:020000040000fa
:08000000e40804000000000008
:020000040000fa
:10040000889fbe008a9fbe00010578000100e000c1
:100410000400350008003c000000e000200032002d
:100420000500370060001000e080180002003b006b
:1004300001f02c001a0037000004be006011b80063
:100440006b0920000982cf00020039000882cf002a
:100450000441b000694252000e00320008003b0027
:1004600082817100610164008904d1000884d30095
:100470008b05e8000442e800f9ff3a000500370068
:100480000804440089844c008b05e9000442e9001b
:10049000fbff3a00540107000af0a70001f0a0009a
:1004a0004f05be004f04be0000000600889fbe003e
:1004b0008a9fbe008c1f780071010700780133000d
:1004c00003866c006450e100240032006420e100e7
:1004d000270032006150e100220032006120e1007b
:1004e000210032008b854200eb07b1000134b800d7
:1004f000003ab8000804420089844a00013ab80072
:100500000030b8008880400009014a000400330030
:100510000000400081804800020149008b05e9008d
:10052000c909dd00830170000100320013002000c2
:10053000c814de004814dd004709de001200b200d6
:10054000c808de00088470002701070001f0a10040
:100550000cf0a70001f0a0005a0137006120e10073
:100560005c0132000801be000200be00f7ff370048
:100570006150e100fcff3a0056013700889fbe0041
:100580008a9fbe008c1f78003d01070044013300a4
:1005900003866c006450e1002e0032006420e1000c
:1005a000330032006150e1002f0032006120e10091
:1005b0003100320085855500eb07b00009002000ae
:1005c00008042000050037000804440089844c001a
:1005d0000a0031000603430087834b0000015300eb
:1005e00081815b00f8ff33000203be000800a00019
:1005f0000804440089844c00f6ff3900c639dd0048
:100600008301730001003200130020008904d1002f
:100610000884d3000998a300050032000800a70051
:100620000300a0008904d1000884d3008b05e800f2
:100630008904d1000884d3000001eb000281d200bc
:10064000e900070001f0a1000cf0a70001f0a000f4
:100650001c0137006420e1001e0132000801be00c9
:100660000200be00f7ff37006120e10019013200ef
:100670006000b800f3ff37000000200001f82700f9
:10068000f0ff370003f0a200889fbe008a9fbe00e3
:100690008c1f7800fa000700010133006450e1006c
:1006a0004f0032006420e1005200320003826c00ef
:1006b00007003b000905d0000306d000820f54005c
:1006c0000c065d000200390002003200890178004a
:1006d000030678008582550004003d000003fd00fc
:1006e0008103fd008502ea008b854200840f7200c1
:1006f00002003b0060001000e08018006011b800ac
:100700000005eb007a28e1000a00390006007800b5
:10071000c75ddd00f707b200878075002d00370048
:10072000828171000a017800610560008180d1003a
:100730000080d3008502e900f9ff3b000604400079
:100740008784480002003b0060041400e0841c0021
:100750000988a300070032008a817100828171003c
:10076000610164008904d1000884d3008b05e8008e
:10077000170037000978a30013003a000b00e000cf
:10078000130034008b05e9000804440089844c0000
:100790000a4474000978a3000d003a000b00e00041
:1007a000070034008b05e9000804440089844c00ec
:1007b00001003a000b0020000978a300f7ff320087
:1007c0000001eb0002003700828171000a0178000d
:1007d000850007000cf0a70001f0a000b900370069
:1007e0006420e10002003a00838f6c00b9003300fe
:1007f0000801be000200be00b20037000001be00ca
:10080000b70007000470a70003f0a1006509b1005c
:10081000160032000d0035006828e10006003500a2
:10082000f0ff2f00f1ff27000300e00013003b0062
:100830000100280000000500000040008180480001
:100840008502e900fcff3a0008003700f88f4200fb
:1008500002003c008000eb00000005008100d10098
:100860000080d3008502e800fcff3a000300e000ae
:1008700002003b0060001000e0801800000006004d
:10088000889fbe008a9fbe008c1f78007c000700f6
:100890001002200002003b0000408800800037006a
:1008a0008a0062006408e10002003a00004088000b
:1008b000880037006108e100fcff32000800be003c
:1008c000030478002dff070001f0a1009900070044
:1008d00008f0a600040037000001be0091042400c7
:1008e000b0fd200067ff070009f0a70001f0a2009b
:1008f00074003700889fbe008a9fbe008c1f78005e
:100900000004be00760007000478a30026003a0029
:100910006120e1002500320009f8a30025003a001b
:100920006420e10021003200f507b1000508a300b2
:100930000200320000004000818048006044b8009e
:1009400003102000020020000000400081804800c9
:100950000805440089854c000a0541008b85490043
:100960000a0550008b855800030033000a00be00c2
:1009700002047400838474008301d1000281d300d7
:10098000830f7100f0ff3a008904d1000884d3007e
:100990006001490082017800c1adde00fb07b000b4
:1009a00011000700470037000960a0000800be00e2
:1009b000440037001202200002408800f0ff2f00a0
:1009c000f1ff27003f0037000001eb00be003700b9
:1009d0000081eb00bc0037000001eb002301370071
:1009e0003200200021013700810020006180550085
:1009f0000b003d000b00200061fe2f000100e10014
:100a00001d00340082817100610164008904d100fd
:100a10000884d3000000e800faff3a0071002000cb
:100a200061006400030070000200600009003200f1
:100a300061044400e0844c000988a50005003200f0
:100a40008b05e8006808e10002003a008904d10043
:100a50000884d300f20f20000258e10005003d0099
:100a6000c75ddd00f907b2008980750008007800d5
:100a7000000006000bf827008b007800000005003e
:100a80000004be00160007000003be000405be00ff
:100a90000200be0012000700844f7500000006002f
:100aa0000200be006450e100050036006420e10051
:100ab000020036000968a30001003a000800be00e9
:100ac0000160a0004f0678004f05be004f04be0035
:100ad00000000600f0ff2f00f1ff2700f9ff3700ac
:100ae000c70ade00f107b200f50fb20008003200bd
:100af000e1cf4200020032000170a0002400050096
:100b0000810f700001003200040805004400050058
:100b1000810f700002003a00140005008502e90010
:100b20000000400081c04800fcff3b000170a000b5
:100b300024000500889fbe008a9fbe008c9fbe00d7
:100b40000004be00e6ff07000800be00890678002a
:100b50006420e10008003900040032000160a000b8
:100b600012022000024088005300370091fc23004d
:100b7000b0fd20004e0037000006eb0009f0a10098
:100b800003f82300020020000800be001e01070039
:100b90000600340001f82300000020000801be0018
:100ba00076fe07000004be002c0020000800be00f6
:100bb00093e82300320a23001301070012003400d7
:100bc0000801be00d1fd2300703d2b00aefe0700e2
:100bd0000005be00b3f32300f27a26000800be0031
:100be00032fe070003f8230002002000a5fe0700e4
:100bf0000801be00a4fe07000a01be005ffe070058
:100c00000004be000c06e8000800be0001f0a100d0
:100c10000200200003982300fb0007000800be002c
:100c2000160035000801be0020fe07000005be00ca
:100c300032cd2c0043fb230093fe0700809fbe00b3
:100c40001269280003d52b000a00be0017fe07001a
:100c5000620f210013ef2b008bfe07000a01be007c
:100c600012fe07004f01be0044fe07000801be004f
:100c70000efe07000801be0083fe07000c00e00026
:100c80000b0032000c10a70001f0a200b2fd200002
:100c900093fc23006260e1000400320022a92000de
:100ca00063f023000c10a70063f8230076fe070012
:100cb0000df0a70001f0a2004f06be004f05be00d8
:100cc0004f04be0000000600889fbe008a9fbe0041
:100cd0008c9fbe00820578000004be0080ff0700e4
:100ce0000800be006420e1000700390002003a005d
:100cf000f1ff2700f0ff2f000160a000120220008a
:100d000002408800550037006120e10003003a00ee
:100d10000b00a70001f823005000370001f0a100ec
:100d20000200210093642400b70007000800be0001
:100d300004003500b2fd2000930c2400b40007002d
:100d40000004be000005eb000b00a6004f0dde0006
:100d500001f0a1000004be0032982f0023ea230016
:100d6000d2fd07000001eb0003f023000b00a700f9
:100d700003f8230044fe0700a0fe07000000a700c0
:100d80000a00a2009efd07000b00e00003003200f5
:100d90000200200003f023003afe070001f0a20049
:100da0000006be000200200093042400bffd0700df
:100db0000801be0034fe0700809fbe000c00be008c
:100dc00022a22a00d3a72300b8fd07004f01be00ce
:100dd0002dfe07000004be0001f0a100020020006b
:100de00003982300880007000800be0019003500a2
:100df0000001be00adfd07000006be00b2c529001f
:100e0000e3622300a9fd070022222b00f3942b00ac
:100e10001dfe07000c01be00a4fd0700e2732800c0
:100e200083c0230018fe07000c01be009ffd0700d1
:100e300042aa2a00a3e22b0013fe07000c01be0009
:100e40009afd07000801be0098fd07000801be00da
:100e50000dfe07000a00a70001f0a2004f06be0029
:100e60004f05be004f04be0000000600889fbe0074
:100e70008a9fbe008c9fbe000206780001f0a7008a
:100e80000cf0a0000004be0015ff07000800be0023
:100e90006420e1000700390002003a00f1ff27005a
:100ea000f0ff2f000160a000120220000240880025
:100eb0005100370009f0a1000800be000200200028
:100ec00003f8230054000700f4ff3c000800be00b4
:100ed00002002000039823004b0007000800be001a
:100ee000300035000200200003f023004a00070014
:100ef00005003c000800be000801be006bfd0700b5
:100f00000005be000e0037000c10a20000002000fb
:100f100001f823000801be00dafd070002002000ee
:100f200003f0230061fd07000005be0071fe07000d
:100f30000200200003002c005cfd07000004be003e
:100f40000a00be00b2d02800130b2c00cefd070013
:100f50000a01be0055fd0700020f2500330b2400d7
:100f6000c9fd0700809fbe000a00be005206220095
:100f700013f02b004dfd0700b2662100f3f62300ad
:100f8000c1fd07000a01be0048fd07004f01be0079
:100f90007afd07000801be0044fd07000801be00fd
:100fa000b9fd07000c00a70007003700b2fd2000c4
:100fb00093fc23000c10a700b3fd07000cf0a70062
:100fc00001f0a2000c0037000cf0a700020037006f
:100fd00001f0a20004003700b2fd200093042400b9
:100fe0000c10a60003003700b2fd200093fc230084
:100ff0000c10a700a4fd07004f06be004f05be0061
:101000004f04be000000060014002000040037005a
:10101000040020001d003700f4ff2f0000003700ff
:10102000889fbe008a9fbe00841f780094fe070040
:101030004f00780011003300f0ff2f00838f6c0009
:1010400006003b00040565000a00a7000800370001
:1010500009f0a6001000200008003700820f54009d
:10106000838f5c00030039001000200001003e0067
:101070000000200009f0a7000000ea004f05be00b4
:101080004f04be000000e00000000600889fbe0084
:101090008a9fbe008c1f78004f26dd0078fe070077
:1010a0007ffe33006120e100430032006250e10026
:1010b00041003e003e0039006420e1003c00320067
:1010c000058255000f003b000402e80038003a009a
:1010d000800f5300818f5b00350034000800be0094
:1010e00003f0a10001f0a60003f0a0000cf0a7009f
:1010f00065fd070073fe37000603430087834b003e
:101100000c4646000005530081855b000200330059
:101110000a03be000c00a0000402e900f6ff3b0039
:10112000850578000602430087824b0004003a00e0
:101130006000b80009f0a70001f0a00061fe3700d0
:101140000002520081825a000704e00004003300cc
:101150000603430087834b008b05e900faff370045
:10116000090578000604be000203be006011b80045
:101170001dfe0700e00f5200e08f5a000700350007
:1011800002003c000c08a300040032000601be006f
:1011900003f0a0000cf0a7003bfd07000a856800e3
:1011a00001f0a1000af0a70001f0a00045fe370001
:1011b0000800be0043fe3700100220000cf0a6001d
:0811c0000040880043fe3700e7
:020000040000fa
:0200000401f009
:04000800fdff0000f8
:020000040000fa
:0200000401f009
:04000c0078ff000079
:020000040000fa
:0200000401f009
:040010007dff000070
:020000040000fa
:0200000401f009
:04001400e7ff000002
:020000040000fa
:0200000401f009
:04001800fcff0000e9
:020000040000fa
:10000800d6450000d6450000d6450000d64500007c
:10001800d6450000d6450000d6450000d64500006c
:1000280024370000863f0000b2410000d64500009a
:10003800d6450000c23f0000be410000da41000082
:10004800d6450000d6450000d6450000d64500003c
:10005800d6450000d645000022420000d6450000e3
:10006800d6450000d6450000d6450000d64500001c
:10007800d6450000d6450000d6450000d64500000c
:10008800d6450000ca410000d6410000d645000010
:10009800ba340000d645000024340000d6450000dc
:1000a800d6450000d6450000d6450000d6450000dc
:1000b800d6450000fe3f00005a4000009640000070
:1000c8000e410000d6450000d6450000d645000088
:1000d800d6450000d6450000d64500001442000071
:1000e800f6410000d6450000d6450000d645000080
:1000f800d6450000d6450000d6450000d64500008c
:10010800d6450000d6450000d6450000d64500007b
:10011800d6450000d6450000d6450000d64500006b
:10012800d6450000d6450000d6450000d64500005b
:10013800d6450000d6450000d6450000d64500004b
:10014800d6450000d6450000d6450000d64500003b
:10015800d6450000d6450000d6450000d64500002b
:10016800d6450000d6450000d6450000d64500001b
:10017800d6450000d6450000d6450000d64500000b
:10018800d6450000d6450000d6450000d6450000fb
:10019800d6450000d6450000d6450000d6450000eb
:1001a800d6450000d6450000d6450000d6450000db
:1001b800d6450000d6450000d6450000d6450000cb
:1001c800d6450000d6450000d6450000d6450000bb
:1001d800d6450000d6450000d6450000d6450000ab
:1001e800d6450000d6450000d6450000d64500009b
:0801f800d6450000d6450000c9
:020000040000fa
:10020800d6450000d6450000d6450000d64500007a
:10021800d6450000d6450000d6450000d64500006a
:1002280024370000863f0000b2410000d645000098
:10023800d6450000c23f0000be410000da41000080
:10024800d6450000d6450000d6450000d64500003a
:10025800d6450000d645000022420000d6450000e1
:10026800d6450000d6450000d6450000d64500001a
:10027800d6450000d6450000d6450000d64500000a
:10028800d6450000ca410000d6410000d64500000e
:10029800ba340000d645000024340000d6450000da
:1002a800d6450000d6450000d6450000d6450000da
:1002b800d6450000fe3f00005a400000964000006e
:1002c8000e410000d6450000d6450000d645000086
:1002d800d6450000d6450000d6450000144200006f
:1002e800f6410000d6450000d6450000d64500007e
:1002f800d6450000d6450000d6450000d64500008a
:10030800d6450000d6450000d6450000d645000079
:10031800d6450000d6450000d6450000d645000069
:10032800d6450000d6450000d6450000d645000059
:10033800d6450000d6450000d6450000d645000049
:10034800d6450000d6450000d6450000d645000039
:10035800d6450000d6450000d6450000d645000029
:10036800d6450000d6450000d6450000d645000019
:10037800d6450000d6450000d6450000d645000009
:10038800d6450000d6450000d6450000d6450000f9
:10039800d6450000d6450000d6450000d6450000e9
:1003a800d6450000d6450000d6450000d6450000d9
:1003b800d6450000d6450000d6450000d6450000c9
:1003c800d6450000d6450000d6450000d6450000b9
:1003d800d6450000d6450000d6450000d6450000a9
:1003e800d6450000d6450000d6450000d645000099
:0803f800d6450000d6450000c7
:020000040000fa
:109800000000000000000000050000000a00000049
:1098100000000000160000000000000069000000c9
:1098200064000000780000000a000000aa030000a5
:10983000aa0300002c030000aa0300007d00000022
:10984000320000000c0000003c000000000000009e
:10985000aa030000410000001400000064000000a2
:10986000190000005000000000000000aa030000e2
:10987000aa0300002c0300001400000000000000f8
:10988000470000001f0700004707000049070000cd
:109890002005000030000000300000003000000013
:1098a0003000000030000000300000000000000028
:1098b00000000000000000000000000000000000a8
:1098c000010000000200000000000000000800008d
:1098d00000080000000800006a0900000a000000fb
:0898e0000a000000ffff000078
:020000040000fa
:1011c8004ff12000007f240000018800000000008b
:1011d800400f020000000000e0012000303a8800c3
:1011e80044e7a90044c7a9004487a9004467a900a7
:1011f8004447a9004427a9004407a900300020005b
:101208003174200082072000a3092000824878005a
:10121800834878008048780010002000217420005e
:101228006204200073052000824878008348780013
:10123800804878002aa3ef002c23ef002023ef003a
:1012480021e3a90021a3a8002183a8002143a80025
:101258002123a9002103a90020e3a80020c3a80096
:1012680020a3a8002063a9002043a9002023a900e7
:1012780023e3a90023c3a90023a3a9002383a9006a
:101288002343a8002323a9002303a90022a3a8001d
:101298002283a9002263a8002243a8002223a900d0
:1012a8002203a900f0f12100201988003223ef0061
:1012b8002623ef002823ef0029e3a90028e3a9004b
:1012c8002963a9002943a9002923a9002903a90002
:1012d8002863a9002843a9002823a9002803a900f6
:1012e8002e23ef00f0ff200080198800aa80a900b3
:1012f800aaa0a900aac0a9008ca3a9008c83a90050
:101308008c23a8008c03a900d0c0b300701c8800ef
:101318009023ef00c0022000901c880000302000bd
:10132800a01c8800b0002000b01c8800ab40a900b9
:10133800ab20a900ab00a90085c0a90000002000cf
:10134800401188002222ef0023e2a90023a2a9006d
:101358002022ef002042a8002022a9009580a900a1
:101368009560a90030102000c011880033e2a90060
:1013780033a2a900b340a800b320a900b300a90074
:101388003022ef003042a9003022a90032e2a90041
:1013980032c2a90097e0a90097c0a900a4c0a8007c
:1013a800a4a0a900a480a8004221ef0010082000f2
:1013b800100a8800a6c0a800a6a0a900a680a800b8
:1013c8004621ef0010082000300a8800b6c0a800a7
:1013d800b6a0a900b680a8004a21ef001008200096
:1013e800500a8800b740a800b720a900b700a80095
:1013f8004e21ef0010082000700a8800b7c0a8002e
:10140800b7a0a900b780a8005221ef00100820005b
:10141800900a8800b840a800b820a900b800a80021
:101428005621ef0020002000b00a8800a540a8003f
:10143800a520a800a500a9008421ef00a740a800c6
:10144800a720a800a700a9008a21ef00b0c0a80023
:10145800b0a0a800b080a9009021ef00b140a8007a
:10146800b120a800b100a9009621ef000622ef00e4
:101478000822ef00ca22ef00d022ef00d622ef00a8
:10148800e222ef00c6a2ef00cca2ef00d2a2ef004a
:10149800dea2ef00cdc2a900cda2a900d202a90008
:1014a800d222a900d242a900d262a900de02a90074
:1014b800de22a9001e21ef002021ef001421ef00f9
:1014c8001821ef0030002000e008880000d4200038
:1014d800d00888001e61a800b240a900b220a80068
:1014e800b200a8008780a9009780a8001021ef000b
:1014f8000621ef00400d23006008880010a1a80015
:1015080084e0a90094e0a900a7c0a800a7a0a800ab
:10151800a780a9001221ef000a21ef00f0ff2f0099
:10152800700888001281a8002c21ef002221ef000a
:1015380090d02300400988002c81a8002ca1a80085
:10154800bbc0a800bba0a800bb80a90089e0a90077
:1015580099e0a8002e21ef002621ef0090d023006b
:10156800500988002ea1a8002e81a800bc40a80020
:10157800bc20a800bc00a9008a00a9009a00a80005
:10158800a440a900a420a800a400a9008200a900e2
:101598008400a9009400a8000421ef000021ef00b6
:1015a80005e1a900580d020000000000704f24005a
:1015b800c05c880000002e00d05c8800704f2400ba
:1015c800e05c880000002e00f05c8800704f24006a
:1015d800e048880000002e00f048880021e2a800ba
:1015e8004c0d02000000000040cf20005061880030
:1015f8008560a90021e2a80087c0a90097c0a800bb
:1016080031e2a8008900a9009900a8008420a90057
:101618009420a80084a0a90094a0a80088a0a900ec
:1016280098a0a80088c0a90098c0a80088e0a900d0
:1016380098e0a8008440a9009440a80084c0a900ac
:1016480094c0a8008720a9009720a8008740a90077
:101658009740a800e202a900e222a90085a0a900fb
:1016680011e1a8002de1a800a03a2000a0498800b7
:10167800100c880040752000b049880030a0200078
:10168800c0498800c0da2000d0498800809b20002b
:101698008000eb003c000800010000000118780001
:1016a8008100e800244302000000000062c9a8008d
:1016b8000b08a9004609a90046a9a9004669a9007e
:1016c8000c28ef00900c200060418800604c8000de
:1016d800030120000300b90043062000110009009f
:1016e8004308d800e0568800d04a80000301200053
:1016f8000300b90043062000110009004308d80080
:10170800a0568800e04a8000030120000300b900c9
:1017180043062000110009004308d800b05688008d
:10172800f04a8000030120000300b90043062000ae
:10173800110009004308d800c0568800004b8000fb
:10174800030120000300b90043062000110009002e
:101758004308d800d0568800d04b8000a05188009c
:10176800030120000300b90043062000110009000e
:101778004308d80070568800604b8000d05188001c
:10178800030120000300b9004306200011000900ee
:101798004308d80060568800e04b80000301200011
:1017a8000300b90043062000110009004308d800cf
:1017b80090568800f04b8000030120000300b90018
:1017c80043062000110009004308d800805688000d
:1017d800804d800003012000110009000380d8001b
:1017e800b04d8800804d8000614d800001005000a0
:1017f8008000eb000002020000000000e34024002b
:1018080002002400be02020000000000c148880057
:10181800d0488800a04d8000012020000181b90037
:10182800d4022000110009004499d800b042880071
:10183800904d8000012020000181b900d4022000d1
:10184800110009004499d800c04288008000eb00cc
:10185800204c80000002020000000000615988004e
:10186800705988008000eb00304b800000020200b5
:101878000000000081598800905988008000eb0022
:10188800504b80000002020000000000c15988008f
:10189800d05988008000eb00a04b800000020200b5
:1018a80000000000e1598800f05988008000eb0032
:1018b800c04b80000002020000000000215a88008e
:1018c800305a88008000eb00404b80000002020084
:1018d80000000000a1598800b05988008000eb0082
:1018e800b04b80000002020000000000015a88008e
:1018f800105a88008000eb00904b80000002020024
:101908000000000041568800505688008000eb0017
:10191800804b800000020200000000000312240037
:10192800020020005602020000000000a15e8800ac
:10193800b05e8800f14c8000e04c8000000202009c
:1019480000000000a3c52400920e2900be02020078
:1019580000000000c1528800b0528800f34c80009b
:10196800e24c8000720e020000000000c1a62000b8
:1019780020c22000a0107800a0107800a0107800e5
:10198800a0107800a0107800a0107800a0107800af
:10199800a0107800700aa9000e0caf00700aa80009
:1019a800114d8000004d8000000202000000000080
:1019b800a3c52400920e2900be0202000000000008
:1019c800e1528800d0528800134d8000024d8000fb
:1019d800720e02000000000021a8200020c2200092
:1019e800a0107800a0107800a0107800a01078004f
:1019f800a0107800a0107800a0107800a01078003f
:101a0800a0107800840aa9000e0caf00840aa80070
:101a18003c89a9006ee9af003c89a8003ca9a9004f
:101a28006f09af003ca9a800414d8000016001008a
:101a3800020037000e0037000d0037005448a80098
:101a48005468a80020002000314d80000100e70004
:101a580009003700000020000100e7005468a900d1
:101a6800100020000100e7005448a90002003700d8
:101a78005448a9005468a9004449a80021e3a800d3
:101a88008de3a8002043a80000000000feff3700f7
:101a9800fa2aef00f82aef00f62aef001fe1a80063
:101aa80013e1a800000006002180200022f1200098
:101ab8008018eb000208e600fdff37000000060072
:101ac800224880000290b9001060880021608800d8
:101ad800324880000290b900022cb400010078005e
:101ae80004acb400424880000290b900022cb40053
:101af8000100780004acb400260e020000000000cb
:101b080010608000605888000000060020488000af
:101b1800b05f8800324880000290b90010608800e9
:101b280021608800424880000290b900022cb4006d
:101b38000100780004acb400260e0200000000008a
:101b480010608000a05f88004148800001f0a70075
:101b5800f42bee00a05f80008000eb0000f0a700ef
:101b68008080eb000002020000000000815d880018
:101b7800905d8800b05f80008000eb0000f0a70057
:101b88008080eb000002020000000000835d8000fe
:101b9800925d80004004020000000000415b880064
:101ba800505b88000000060030488000b05f880065
:101bb800224880000290b9001060880021608800e7
:101bc800424880000290b900022cb400010078005d
:101bd80004acb400260e0200000000001060800073
:101be800a05f88004148800001f0a700f42bee00b8
:101bf800a05f80008000eb0000f0a7008080eb0071
:101c08000002020000000000815d8800905d8800ed
:101c1800b05f80008000eb0000f0a7008080eb0040
:101c28000002020000000000835d8000925d8000d9
:101c38004004020000000000615b8800705b8800bf
:101c480000000600048cd6004200af000000060029
:101c5800dc0e020000000000e60e0200000000009a
:101c680000012000f05f88000aacd6000cacd6005a
:101c780006acd60008acd6000aacd6000cacd60030
:101c880006acd60008acd6004200a80002acd600cc
:101c980004acd60020608000080cb50002003a00b1
:101ca80010608000060cb500050039001060800047
:101cb800062cb5002060800008acb500022ca800f6
:101cc800020ca900fe2bed00e7ff3a004200a90034
:101cd80004acd70002acd70000000600fc2bef00d4
:101ce800f00e0200000000004200af0000000600f5
:101cf800280f02000000000000022000f05f8800aa
:101d08000281d2008381d20026c220000900080087
:101d180006000000168bd200a00020009600780074
:101d2800008050004200af00000b780026007800c9
:101d3800fe2bed00f2ff3a00fc0baf000e0ca800e2
:101d48004200a90000000600e05f880000022000b1
:101d5800f05f880002c12000a00020004200a90016
:101d6800e15f800001800800020000004200af002f
:101d7800120940001299d30004acd70002acd70076
:101d8800fe2bed00f3ff3a0042007800f1ff2f0030
:101d9800008040004200ae00048cd6004200af0034
:101da800000006000e0caf000e0007000000060041
:101db80010608000506088002060800060608800ab
:101dc80000000600062cef00082cef00022cef00a4
:101dd800042cef00000006000380d2004200ae0091
:101de800000006002060800001002800010060005b
:101df80002acee0004acee00022cec0001003a004c
:101e0800042cec00fc2bec00040cb40000000600d1
:101e1800088cd6004200ae0000000600406080003a
:101e2800010028000100600006acee0008acee00de
:101e3800062cec0001003a00082cec00fc2bec000e
:101e4800080cb400000006000e2cef00102cef0068
:101e5800122cef00142cef00162cef00182cef00ba
:101e68001a2cef001c2cef001e2cef00202cef008a
:101e7800222cef00000006000000eb0000077800ad
:101e88000c000900002f78000007eb000000060096
:101e9800204d8000310020000180e7001900370044
:101ea80020418000410620006f29af00010040005a
:101eb8006f29ae0001005000c14420000180e600f7
:101ec8006f29a90041bb2f000100e6006f29a80077
:101ed80020418800005f88006f49af002828ec0087
:101ee8006f49ae002828ed004041800061092000bc
:101ef8000180e6006f49a900210320000100e600e7
:101f08006f49a800515a8000605a800003122400cb
:101f1800020020005602020000000000fe0302003a
:101f28000000000002a02000015020000180e6000f
:101f380002005000705a8800c15e8000d05e8000a8
:101f480003122400020020005602020000000000d4
:101f5800fe0302000000000002a020000150200043
:101f68000180e60002005000e05e8800705a8000a0
:101f7800e15e8000234d8000320020000218e70057
:101f8800015f80000218e7000000eb00010050002c
:101f9800800178000150200002a020000180e600a6
:101fa800820150008100ea000100e6008201400041
:101fb800235b8800a4002000110009008401d800d8
:101fc80030418800205b8000115f8000105f88002e
:101fd80001005000800178000150200002a020007c
:101fe8000180e600820150008100ea000100e6005d
:101ff80082014000c354880023448800224b80009b
:102008006a11b800235b8000030078000298e6009c
:10201800020078000201ea000218e60002007800d7
:10202800205b8800104488005408af00bc0a3700c1
:10203800205b8000011420000180e6003c2aef00ac
:102048000180e600100037008100ea000100e60088
:102058003c2aef000100e6000b003700205b8000ff
:10206800e15180000100400080017800429c20007e
:102078000298e600020078000201ea000218e60071
:1020880002007800e0518800205b80008000eb00af
:1020980000f0a7008080eb000002020000000000b2
:1020a800a33f240002002000be020200000000003e
:1020b80083598000925980005602020000000000f7
:1020c8006155880070558800c05480008000eb007e
:1020d80000f0a7008080eb00000202000000000072
:1020e800831c240002002000be0202000000000041
:1020f800a3598000b2598000560202000000000077
:102108008155880090558800e05180008000eb00e0
:1021180000f0a7008080eb00000202000000000031
:10212800c361240002002400be0202000000000077
:10213800c3598000d25980005602020000000000f6
:10214800a1558800b05588006355800072558000fd
:10215800440302000000000083558000925580006f
:1021680044030200000000006e69af0001f0a20005
:10217800fe0302000000000000448800000278000e
:10218800624b80000200400080017800614b8000b3
:10219800c10bb000624b8000c20bb1000180e600a9
:1021a800810178000200e60082017800d35188009e
:1021b8000400780000f0a7000000ea008000eb00af
:1021c8000002020000000000833424000200200006
:1021d800be02020000000000235a8000325a80002c
:1021e8005602020000000000215688003056880080
:1021f800804b80006a00b80001598000234d8000a0
:10220800320020000218e700414180000100500020
:10221800e0548800914b80008100ea000100e6004c
:102228009c2aef00f24b80000100e600f24a800091
:10223800b2518800e0548000f1548000f0548800c6
:102248000100500080017800022820000298e60072
:10225800020078000201ea000218e6000200780095
:1022680050558800924b8000e354800003007800aa
:102278000298e600020078000201ea000218e6006f
:1022880002007800e05488005408af00370a37008d
:10229800e05480008000eb0000f0a7008080eb0095
:1022a8000002020000000000832424000200200035
:1022b800be02020000000000e3598000f2598000cd
:1022c8005602020000000000c1558800d055880061
:1022d800505580008000eb0000f0a7008080eb00e4
:1022e8000002020000000000831c240002002000fd
:1022f800be02020000000000035a8000125a80004b
:102308005602020000000000e1558800f0558800e0
:10231800c3558000d455800044030200000000002b
:10232800235680003256800044030200000000005b
:102338006e09af0001f0a200fe03020000000000d9
:10234800d24b80000200400080017800d14b800011
:10235800c10bb000d24b8000c20bb1000180e60077
:10236800810178000200e60082017800a35188000c
:10237800e04b8000c05188000000060022212000a8
:10238800f04480000200e600f2448800d044800057
:102398000200e600d2448800104580000200e600f2
:1023a80012458800304580000200e600324588006a
:1023b800f2552000f04480000280e600f2448800d4
:1023c800d04480000280e600d24488001045800096
:1023d8000280e60012458800304580000280e60051
:1023e800324588003d29af000700370046c9ae00d6
:1023f800050037004449af0046c9a9000000eb00ba
:102408004449af0010438800104380003100200089
:102418000100e6000400370020438000e1002000ae
:102428000100e70000000600204d80002100200088
:102438000180e600020037003c49a9003c69a90078
:102448000800fc00204d8000410020000180e600cb
:102458000700370000007800050033000060010025
:1024680003003700240037003300370032003700fc
:102478006ea9a9004449ae000d0037000f00fc000a
:10248800d14a8000a1498800e04a800081004000cc
:10249800b1498800f04a800081004000c1498800a5
:1024a800004b800081004000d149880000000600f0
:1024b8006ea9a90046c9af003b0037000c48af0021
:1024c800eeff37000b00fc00d1448000a1498800d2
:1024d800f044800081004000b14988001045800028
:1024e80081004000c14988003045800081004000db
:1024f800d1498800000006004449ae00ecff3700cf
:102508006ea9a8000f00fc00a1518000a149880015
:10251800c051800081004000b1498800b05180005e
:1025280081004000c1498800d051800081004000ee
:10253800d1498800000006004449af00ccff3700ad
:1025480046c9af00180037001a00fc00a1518000ee
:102558003c69ae00d1448000a14988000001eb002d
:10256800f04480000200e600e04a8000810040005c
:10257800b1498800104580000200e600f04a80005a
:1025880081004000c1498800d05180003c49ae001c
:10259800304580000200e600004b800081004000ca
:1025a800d1498800000006000f00fc00714580003a
:1025b800a14988008045800081004000b149880019
:1025c8009045800081004000c1498800a0458000f6
:1025d80081004000d149880000000600c04a800000
:1025e8000000e00004003200815a80004409a9007c
:1025f8000008e6004409a800504a80000000e000f6
:1026080004003200515980004429a9000008e6005e
:102618004429a800944a8000a50020000520b9009c
:10262800714880004489a9000008e6004489a80090
:1026380081488000c01220000008e600040037002e
:102648004042200044a9a9000008e60044a9a800c7
:102658005009e2000f003200844a8000431f200026
:102668000320b900e35a8000f25a800044c9a90047
:102678000198e60001003700060037000118e7005e
:102688000200370044c9a800020037000090e600a5
:1026980044c9a800704a8000017d20000102b900e9
:1026a8008000eb004206200011000900422ad800f1
:1026b800b248800002034000704a800041062000b2
:1026c8000102b90044e9a90004b0e60044e9a80001
:1026d8004609ae0000000600a0488000c112200094
:1026e8000180e60046a9a9000c68af000e0037007b
:1026f800805a8000a10020004629af006100200018
:102708000100e60000000600005980004101200099
:102718004629af00110420000100e6000000060071
:102728000c68a80046a9a900805a80005100200022
:102738004629af00310020000180e60000000600b5
:1027480000598000410120004629af0011042000f3
:102758000180e6000000060046a9a8000c68a90050
:10276800000006004449af002028ef002028ec00b4
:1027780001418000900020000008e6004400370076
:10278800a000200000418800204d8000210020008a
:102798000180e7003c2aef00c0448000c10d200002
:1027a8000180e6003a003700b0458000c10d2000e6
:1027b8000180e60036003700b045800001052000a2
:1027c8000100e60032003700c0448000910b200071
:1027d8000100e600750037006a08e20006003a00ca
:1027e800b0458000910b20000180e6002a003700e8
:1027f8006a28ec00280037006828ef006a28ec00f7
:1028080050438000510020000100e60022003700fc
:102818006228ec00204d8000110020000180e600b5
:1028280006003a0046c9a900104380004100200074
:102838000180e6006228ef00150037001043800091
:10284800510020000180e6006228ef0046c9a90077
:10285800410020000100e70046c9a8000100e70088
:102868003d29a900410020000180e7000800370049
:10287800d044800070458800f0448000804588007e
:10288800104580009045880030458000a0458800ac
:102898006828ef006a28ef00c0448000b04588002f
:1028a80046c9ae00000006004449af00000006001b
:1028b8003d09a80070458000e003b000d1448000c5
:1028c8000088e6001500370070458000e003b1007d
:1028d800d14480000008e60019003700a0458000b8
:1028e800e003b000314580000088e6001d00370095
:1028f800a0458000e003b100314580000008e600f3
:10290800210037005a28ef005c28ef005e28ef000e
:102918006028ef003d09a900000006005a28ec00d5
:10292800d0428000e10120000180e6009b003700d2
:102938005c28ef005e28ef006028ef00000006002a
:102948005c28ec00e0428000e10120000180e60004
:10295800b00037005a28ef005e28ef006028ef002b
:10296800000006005e28ec00f0428000e101200033
:102978000180e6009c0337005a28ef005c28ef002e
:102988006028ef00000006006028ec00004380008b
:10299800e10120000180e600340337005a28ef00e7
:1029a8005c28ef005e28ef00000006006a28ef00b0
:1029b80046c9af00b6ff3700c04480007108200048
:1029c8000180e600b2ff37006808e20006003a001e
:1029d800b0458000710820000100e600acff370018
:1029e8006828ec00acff3700c0448000a105200037
:1029f8000100e600a6ff37006828ec00404380008d
:102a0800f10020000100e600a3ff3700482aec008f
:102a180040528000310020000180e600482aef0083
:102a28003c2aef00604b8000d05188003c49a90047
:102a38003c69a90040528000110020000100e70015
:102a48003c49a800210020000100e7003c69a800db
:102a58003c89ae003c49a9003ca9ae003c69a900ec
:102a6800204d8000210020000180e60088ff37000b
:102a78005408ae0086ff37005408ae0084ff3700c4
:102a880020002000414d80000180e700030037004e
:102a98005448aa005468aa00060037000000200025
:102aa800414d80000180e700020037005448a8002b
:102ab8005468a80020002000314d80000100e70084
:102ac80006003700000020000100e7005468a90054
:102ad800100020000100e7005448a9003c49a90063
:102ae8003c69a9006aff3700a04380009143800039
:102af8000008e700000006004669a9007408e20023
:102b080060003a0090438000410920000180e700fe
:102b18000d00370046c9af0046c9a9003c09a90005
:102b28003c29a9004a2aef004c2aef004e2aef0060
:102b38006228ec0010438000510020000100e700eb
:102b48006228ef004f00370010438000e40068005f
:102b58004c003a0090438000010920000180e70002
:102b6800190037003c09a90046c9af000b0037001f
:102b78004a0ae20047003a004c0ae20029013a00fa
:102b88004e0ae20098013a006428ed003d003b003f
:102b9800d0012000204388003a0037005c28ef006d
:102ba8005a28ef005e28ef006028ef006628ed0045
:102bb80034003b00200120005408af00d001200061
:102bc800304388002f00370090438000110920000f
:102bd8000180e7001b0037003c09a90046c9af0087
:102be8000c0037004a0ae2009c003a004c0ae20056
:102bf800f9013a004e0ae20045023a006428ec0066
:102c080020438000e10120000100e7006428ef0074
:102c18001c0037005c28ef005a28ef005e28ef0000
:102c28006028ef006628ec00304380003101200066
:102c38005408af00e10120000180e6006628ef009b
:102c48001000370090438000210920000180e70030
:102c58000400370046c9af00840237005a05370020
:102c68000800370090438000310920000180e70008
:102c78000400370046c9af00db023700ad05370056
:102c8800000037003d09a90090438000a043880058
:102c98000000060050528000110020000180e7006b
:102ca8000f0037008e29ec00704c8000c105200011
:102cb800020320000180e600724c88001104200005
:102cc8000180e600efff3700910320000100e600d5
:102cd800ecff370012042000724c8800e9ff37002f
:102ce800210020000180e7000f0037009029ec0048
:102cf800804c8000c1052000020320000180e6000e
:102d0800824c8800110420000180e600ddff3700b6
:102d1800910320000100e600daff370012042000ca
:102d2800824c8800d7ff3700310020000180e7007f
:102d38000f0037009229ec00904c8000c10520005c
:102d4800020320000180e600924c88001104200054
:102d58000180e600cbff3700910320000100e60068
:102d6800c8ff370012042000924c8800c5ff3700c6
:102d7800410020000180e7000f0037009429ec0093
:102d8800a04c8000c1052000020320000180e6005d
:102d9800a24c8800110420000180e600b9ff37002a
:102da800910320000100e600b6ff3700120420005e
:102db800a24c8800b3ff3700510020000180e700d3
:102dc8000f0037009629ec00b04c8000c1052000a8
:102dd800020320000180e600b24c880011042000a4
:102de8000180e600a7ff3700910320000100e600fc
:102df800a4ff370012042000b24c8800a1ff37005e
:102e0800610020000180e7000f0037009829ec00de
:102e1800c04c8000c1052000020320000180e600ac
:102e2800c24c8800110420000180e60095ff37009d
:102e3800910320000100e60092ff370012042000f1
:102e4800c24c88008fff3700710020000180e70026
:102e58008cff37006ec9aa008aff370050528000e5
:102e6800110020000180e7000f0037008e29ed00d7
:102e7800704c8000f1022000b20520000100e6003d
:102e8800724c8800910320000100e6007dff3700a6
:102e9800110420000180e6007aff37009203200029
:102ea800724c880077ff3700210020000180e7007e
:102eb8000f0037009029ed00804c8000f1022000bf
:102ec800b20520000100e600824c88009103200032
:102ed8000100e6006bff3700110420000180e600c6
:102ee80068ff370092032000824c880065ff370096
:102ef800310020000180e7000f0037009229ed0023
:102f0800904c8000f1022000b20520000100e6008c
:102f1800924c8800910320000100e60059ff370019
:102f2800110420000180e60056ff370092032000bc
:102f3800924c880053ff3700410020000180e700d1
:102f48000f0037009429ed00a04c8000f10220000a
:102f5800b20520000100e600a24c88009103200081
:102f68000100e60047ff3700110420000180e60059
:102f780044ff370092032000a24c880041ff37002d
:102f8800510020000180e7000f0037009629ed006e
:102f9800b04c8000f1022000b20520000100e600dc
:102fa800b24c8800910320000100e60035ff37008d
:102fb800110420000180e60032ff37009203200050
:102fc800b24c88002fff3700610020000180e70025
:102fd8000f0037009829ed00c04c8000f102200056
:102fe800b20520000100e600c24c880091032000d1
:102ff8000100e60023ff3700110420000180e600ed
:1030080020ff370092032000c24c88001dff3700c4
:10301800710020000180e7001aff37006ec9aa007e
:1030280018ff370060528000110020000180e7007f
:10303800060037005e2aec00a1002000f052800054
:103048000180e6005e2aef004b00370060528000e6
:10305800210020000180e70006003700602aec000c
:10306800a1002000005380000180e600602aef00e4
:103078004100370060528000310020000180e700e5
:1030880006003700622aec00a100200010538000df
:103098000180e600622aef003700370060528000a6
:1030a800410020000180e70006003700642aec0098
:1030b800a1002000205380000180e600642aef0070
:1030c8002d00370060528000510020000180e70089
:1030d80006003700662aec00a1002000305380006b
:1030e8000180e600662aef00230037006052800066
:1030f800610020000180e70006003700682aec0024
:10310800a1002000405380000180e600682aef00fb
:103118001900370060528000710020000180e7002c
:10312800060037006a2aec00a100200050538000f6
:103138000180e6006a2aef000f0037006052800025
:10314800810020000180e700060037006c2aec00af
:10315800a1002000605380000180e6006c2aef0087
:103168000500370060528000910020000180e700d0
:10317800c4fe3700700aaa0080538000706088007f
:10318800e0a5200001c12000b0187800b018780030
:10319800b0187800b0187800b0187800b018780027
:1031a800b0187800b018780070002000a80e02004f
:1031b8000000000021608000f14c88001060800051
:1031c800e04c88000002020000000000a3c52400b3
:1031d800920e2900be02020000000000c1528800c1
:1031e800b0528800a7fe37007052800011002000fe
:1031f8000180e70006003700722aec002100200059
:10320800905380000180e600722aef0055003700d5
:1032180070528000210020000180e700060037007e
:10322800742aec00a1002000a05380000180e60071
:10323800742aef004b0037007052800031002000e4
:103248000180e70006003700762aec00a100200084
:10325800b05380000180e600762aef004100370075
:1032680070528000410020000180e700060037000e
:10327800782aec00a1002000c05380000180e600fd
:10328800782aef0037003700705280005100200084
:103298000180e700060037007a2aec00a100200030
:1032a800d05380000180e6007a2aef002d00370015
:1032b80070528000610020000180e700060037009e
:1032c8007c2aec00a1002000e05380000180e60089
:1032d8007c2aef0023003700705280007100200024
:1032e8000180e700060037007e2aec00a1002000dc
:1032f800f05380000180e6007e2aef0019003700b5
:1033080070528000810020000180e700060037002d
:10331800802aec00a1002000005480000180e60013
:10332800802aef000f0037007052800091002000c3
:103338000180e70006003700822aec00a100200087
:10334800105480000180e600822aef000500370053
:1033580070528000a10020000180e70049fe37007c
:10336800840aaa00205480007060880020a72000ea
:1033780001c12000b0187800b0187800b0187800a3
:10338800b0187800b0187800b0187800b018780035
:10339800b0187800b018780080002000a80e02004d
:1033a8000000000021608000114d8800106080003e
:1033b800004d88000002020000000000a3c52400a0
:1033c800920e2900be02020000000000e1528800af
:1033d800d05288002bfe3700605280001100200078
:1033e8000180e700050037005e2aed0062ff3b0020
:1033f80093002000f35288005fff3700605280007e
:10340800210020000180e70005003700602aed0058
:1034180059ff3b00930020000353880056ff3700f4
:1034280060528000310020000180e700050037006d
:10343800622aed0050ff3b009300200013538800e0
:103448004dff370060528000410020000180e700f6
:1034580005003700642aed0047ff3b009300200079
:103468002353880044ff3700605280005100200039
:103478000180e70005003700662aed003eff3b00ab
:1034880093002000335388003bff370060528000d0
:10349800610020000180e70005003700682aed0080
:1034a80035ff3b00930020004353880032ff37006c
:1034b80060528000710020000180e700050037009d
:1034c8006a2aed002cff3b0093002000535388002c
:1034d80029ff370060528000810020000180e7004a
:1034e800050037006c2aed0023ff3b009300200005
:1034f8006353880020ff370060528000910020004d
:103508000180e700dffd3700700aaa001aff3700c4
:1035180070528000110020000180e700050037008c
:10352800722aed008fff3b001300200093538800a0
:103538008cff370070528000210020000180e700d6
:1035480005003700742aed0086ff3b009300200039
:10355800a353880083ff3700705280003100200099
:103568000180e70005003700762aed007dff3b006b
:1035780093002000b35388007aff37007052800010
:10358800410020000180e70005003700782aed009f
:1035980074ff3b0093002000c353880071ff37007d
:1035a80070528000510020000180e70005003700bc
:1035b8007a2aed006bff3b0093002000d35388006c
:1035c80068ff370070528000610020000180e7002a
:1035d800050037007c2aed0062ff3b0093002000c5
:1035e800e35388005fff37007052800071002000ad
:1035f8000180e700050037007e2aed0059ff3b00f7
:1036080093002000f353880056ff37007052800063
:10361800810020000180e70005003700802aed00c6
:1036280050ff3b0093002000035488004dff3700f3
:1036380070528000910020000180e70005003700eb
:10364800822aed0047ff3b009300200013548800b6
:1036580044ff370070528000a10020000180e7007d
:1036680088fd3700840aaa003eff37005c28ef0077
:103678005a28ef005e28ef006028ef0030438000f2
:103688000000e000b700320030438000e10068002d
:10369800ba00320030438000e2006800c300320004
:1036a80030438000e3006800cc00320030438000e3
:1036b800e4006800d500320030438000e50068006f
:1036c800fa00320030438000e6006800f90032005a
:1036d80030438000e7006800060132003043800074
:1036e800e80068000f01320030438000e9006800fc
:1036f8001801320030438000ea00680021013200de
:1037080030438000eb0068002a013200304380001b
:10371800ec0068003b01320030438000ed00680097
:103728006c02320030438000ee0068007b023200f9
:1037380030438000ef0068008a0232003043800086
:10374800f00068008c02320030438000f10068000d
:103758008e02320030438000f20068008c01320093
:1037680030438000f30068008e013200304380004f
:10377800f40068008d01320030438000f5006800d5
:103788008c01320030438000f60068008b01320063
:1037980030438000f70068008a013200304380001f
:1037a800f80068008901320030438000f9006800a1
:1037b8009d01320030438000fa006800ad013200fc
:1037c80030438000fb006800c301320030438000b2
:1037d800fc006800d901320030438000fd00680019
:1037e800f001320027fd37005c28ef005a28ef006f
:1037f8005e28ef006028ef00304380000000e00002
:103808000201320030438000e10068000401320008
:1038180030438000e20068000c0132003043800031
:10382800e30068001401320030438000e4006800bf
:103838007600320030438000e50068009b003200cb
:1038480030438000e60068001601320030438000f3
:10385800e70068002201320030438000e800680079
:103868002a01320030438000e9006800320132004a
:1038780030438000ea0068003a013200304380009b
:10388800eb006800cb00320030438000ec00680099
:10389800dc00320030438000ed0068000d02320089
:1038a80030438000ee0068001c0232003043800084
:1038b800ef0068002b02320030438000f0006800ff
:1038c8002d02320030438000f100680037023200d8
:1038d80030438000f20068002d0132003043800040
:1038e800f30068002f01320030438000f4006800c4
:1038f8002e01320030438000f50068002d013200af
:1039080030438000f60068002c013200304380000c
:10391800f70068002b01320030438000f80068008f
:103928003601320030438000f90068003e01320061
:1039380030438000fa0068005b01320030438000a9
:10394800fb0068007101320030438000fc00680011
:10395800ae01320030438000fd006800c40132002f
:10396800c8fc37006429ec0071092000204b800056
:103978000180e6006429ef00c2fc37006629ec00ec
:1039880071092000304b80000180e6006629ef00b5
:103998008000eb00304b80000002020000000000b5
:1039a8008159880090598800b6fc37006829ec00d6
:1039b80071092000404b80000180e6006829ef0073
:1039c8008000eb00404b8000000202000000000075
:1039d800a1598800b0598800aafc37006a29ec0070
:1039e80071092000504b80000180e6006a29ef0031
:1039f8008000eb00504b8000000202000000000035
:103a0800c1598800d05988009efc3700a041800029
:103a1800604d88005428ae0006003700d041800071
:103a2800804d880003012000110009000380d800a0
:103a3800b04d8800804d8000614d8000010050002d
:103a48008000eb000002020000000000e3402400b8
:103a580002002400be02020000000000c1488800e5
:103a6800d0488800304580003d09af00a04580005f
:103a7800604b8800222120000200e600624b88008b
:103a8800f25520000280e600624b8800604b8000ff
:103a9800030120000300b9004306200011000900bb
:103aa8004308d8006056880076fc37006e69aa0083
:103ab80074fc37007029ec00910c2000804b8000ca
:103ac8000180e6007029ef008000eb00804b800049
:103ad800000202000000000003122400020020007f
:103ae8005602020000000000a15e8800b05e880057
:103af80064fc37007229ec00910c2000904b800088
:103b08000180e6007229ef008000eb00904b8000f6
:103b1800000202000000000041568800505688004c
:103b280058fc37007429ec0071092000a04b800074
:103b38000180e6007429ef008000eb00a04b8000b4
:103b48000002020000000000e1598800f0598800d6
:103b58004cfc37007629ec0071092000b04b80003e
:103b68000180e6007629ef008000eb00b04b800072
:103b78000002020000000000015a8800105a880064
:103b880040fc37007829ec0071092000c04b800008
:103b98000180e6007829ef008000eb00c04b800030
:103ba8000002020000000000215a8800305a8800f4
:103bb80034fc370070418000504d8800d0448000ac
:103bc8003d09af0070458000d04b880022212000bd
:103bd8000200e600d24b8800f25520000280e60081
:103be800d24b8800d04b8000030120000300b900ad
:103bf80043062000110009004308d80070568800c9
:103c080020fc37006e09aa001efc37006429ed006d
:103c180002003b0063092000234b880019fc370091
:103c28006629ed0002003b0063092000334b880041
:103c38008000eb00304b8000000202000000000012
:103c480081598800905988000efc37006829ed00da
:103c580002003b0063092000434b88008000eb0012
:103c6800404b80000002020000000000a1598800bb
:103c7800b059880003fc37006a29ed0002003b00b8
:103c880063092000534b88008000eb00504b8000f4
:103c98000002020000000000c1598800d0598800c5
:103ca800f8fb37007029ed0002003b00830c200070
:103cb800834b88008000eb00804b800000020200ec
:103cc8000000000003122400020020005602020037
:103cd80000000000a15e8800b05e8800e9fb3700a4
:103ce8007229ed0002003b00830c2000934b8800f2
:103cf8008000eb00904b80000002020000000000f2
:103d08004156880050568800defb37007429ed00c4
:103d180002003b0063092000a34b88008000eb00f1
:103d2800a04b80000002020000000000e15988005a
:103d3800f0598800d3fb37007629ed0002003b00dc
:103d480063092000b34b88008000eb00b04b800073
:103d58000002020000000000015a8800105a880082
:103d6800c8fb37007829ed0002003b0063092000fa
:103d7800c34b88008000eb00c04b800000020200ab
:103d880000000000215a8800305a8800bdfb370027
:103d98003d09af00bbfb37003d29a90046c9a90072
:103da800b8fb37008289aa00b6fb37008269aa00ef
:103db800b4fb37008209aa00b2fb37008229aa00a7
:103dc800b0fb37008249aa00aefb37008429ec001b
:103dd80071092000204c80000180e6008429ef0052
:103de8008000eb00204c8000000202000000000070
:103df8006159880070598800a2fb37008429ed00ba
:103e080002003b0063092000234c88008000eb007f
:103e1800204c800000020200000000006159880068
:103e28007059880097fb3700d0418000804d88008a
:103e380003012000110009000380d800b04d88005c
:103e4800804d8000614d8000010050008000eb0033
:103e58000002020000000000e340240002002400e9
:103e6800be02020000000000c1488800d048880057
:103e780084fb3700b429ec0091022000a04d80009b
:103e88000180e600b429ef00a04d80000120200049
:103e98000181b900d4022000110009004499d8001a
:103ea800b042880077fb3700b429ed0002003b00e0
:103eb80083022000a34d8800a04d8000012020002f
:103ec8000181b900d4022000110009004499d800ea
:103ed800b04288006bfb3700b229ec009102200049
:103ee800904d80000180e600b229ef00904d8000df
:103ef800012020000181b900d4022000110009002e
:103f08004499d800c04288005efb3700b229ed0012
:103f180002003b0083022000934d8800904d8000f2
:103f2800012020000181b900d402200011000900fd
:103f38004499d800c042880052fb3700a629ec00fb
:103f480031002000304d80000180e600a629ef00f6
:103f5800414d800001600100020037000e0037006b
:103f68000d0037005448a8005468a800200020001d
:103f7800314d80000100e70042fb370000002000bf
:103f88000100e7005468a900100020000100e700c4
:103f98005448a9003bfb37005448a9005468a900bd
:103fa80038fb3700a829ec0031002000404d800084
:103fb8000180e600a829ef00414d80000160010062
:103fc800020037000e0037000d0037005448a800e3
:103fd8005468a80020002000314d80000100e7004f
:103fe80028fb3700000020000100e7005468a90002
:103ff800100020000100e7005448a90021fb370009
:104008005448a9005468a9001efb3700a629ed00f2
:1040180002003b0023002000334d8800414d800002
:1040280001600100020037000e0037000d00370064
:104038005448a8005468a80020002000314d800092
:104048000100e7000ffb3700000020000100e70037
:104058005468a900100020000100e7005448a90096
:1040680008fb37005448a9005468a90005fb37002d
:10407800a829ed0002003b0023002000434d8800e2
:10408800414d800001600100020037000e0037003a
:104098000d0037005448a8005468a80020002000ec
:1040a800314d80000100e700f6fa370000002000db
:1040b8000100e7005468a900100020000100e70093
:1040c8005448a900effa37005448a9005468a900d9
:1040d800ecfa3700104580003d09af00904580009c
:1040e800f04b8800222120000200e600f24b8800f5
:1040f800f25520000280e600f24b8800f04b800069
:10410800030120000300b900430620001100090044
:104118004308d80080568800dafa3700f044800057
:104128003d09af0080458000e04b88002221200037
:104138000200e600e24b8800f25520000280e6000b
:10414800e24b8800e04b8000030120000300b90027
:1041580043062000110009004308d8009056880043
:10416800c8fa37003c89aa006ee9a9003c89af006b
:104178006ee9a800c3fa37003ca9aa006f09a90094
:104188003ca9af006f09a800befa37003d09af008f
:10419800bcfa3700a429ec00204d80004100200023
:1041a8000180e600a429ef00b6fa37003d09af0008
:1041b800b4fa3700a429ed00b2fa3b003000200021
:1041c800204d8800affa3700204380000000e0004f
:1041d800bf01320020438000e1006800b3003200d4
:1041e80020438000e2006800bb00320020438000ca
:1041f800e3006800c300320020438000e400680048
:10420800c100320020438000e5006800c900320088
:1042180020438000e6006800d1003200204380007f
:10422800e7006800d900320020438000e8006800f9
:10423800e400320020438000e9006800ec0032000e
:1042480020438000ea0068005701320020438000c4
:10425800eb0068005601320020438000ec00680043
:104268006501320020438000ed0068006e013200d5
:1042780020438000ee0068008c013200204380005b
:10428800ef0068008600320020438000f0006800dc
:104298004901320020438000f1006800e20032004a
:1042a80020438000f2006800ef00320020438000c5
:1042b800f3006800fc00320020438000f40068002e
:1042c8000901320020438000f500680061013200d6
:1042d80020438000f600680064013200204380001b
:1042e800f70068001801320020438000f8006800d9
:1042f8001701320020438000f900680016013200df
:1043080020438000fa006800150132002043800035
:10431800fb0068001801320020438000fc006800a0
:104328001701320020438000fd0068001a013200a6
:1043380054fa3700204380000000e0006401320096
:1043480020438000e10068005e00320020438000c6
:10435800e20068006600320020438000e300680045
:104368006800320020438000e40068006c003200de
:1043780020438000e500680074003200204380007c
:10438800e60068007c00320020438000e7006800f7
:104398008500320020438000e80068008f0032006a
:1043a80020438000e9006800980032002043800024
:1043b800ea006800fc00320020438000eb0068003f
:1043c800fb00320020438000ec006800110132003d
:1043d80020438000ed00680019013200204380006e
:1043e800ee0068003101320020438000ef006800d1
:1043f8002b00320020438000f0006800ee003200fd
:1044080020438000f10068008700320020438000cc
:10441800f20068009400320020438000f300680036
:10442800a100320020438000f4006800ae00320092
:1044380020438000f500680012013200204380000c
:10444800f60068001401320020438000f70068007d
:10445800bd00320020438000f8006800bc00320034
:1044680020438000f9006800bb0032002043800030
:10447800fa006800ba00320020438000fb006800a0
:10448800bd00320020438000fc006800bc00320000
:1044980020438000fd006800bf003200f9f93700b2
:1044a8004629aa0046a9a900f6f937004829ec00d0
:1044b80051062000404a80000180e6004829ef00ac
:1044c800f0f937004829ed00eef93b0043062000db
:1044d800434a8800ebf937004a29ec00e102200042
:1044e800504a80000180e6004a29ef00e5f93700cc
:1044f8004a29ed00e3f93b00d3022000534a880023
:10450800e0f937000000fe004c29ec0051002000c3
:10451800604a80000180e6004c29ef00d9f9370095
:104528004c29ed00d7f93b0043002000634a88007e
:10453800d4f937004e29ec0051062000704a80005b
:104548000180e6004e29ef00cef937004e29ed0034
:10455800ccf93b0043062000734a8800c9f93700ac
:104568005029ec0051062000804a80000180e600b6
:104578005029ef00c3f937005029ed00c1f93b007d
:1045880043062000834a8800bef937005229ec0010
:10459800b10f2000904a8000c30320000180e6008c
:1045a800934a8800b7f937005229ed00b10320007b
:1045b800904a8000a30f20000100e600934a88007b
:1045c800b0f937005429ec0051062000a04a8000b9
:1045d8000180e6005429ef00aaf937005429ed00bc
:1045e800a8f93b0043062000a34a8800a5f9370034
:1045f80056a9ec00f1152000b04a8000a305200060
:104608000180e600b34a88009ef9370056a9ed00fc
:1046180091052000b04a8000e31520000100e60063
:10462800b34a880097f93700d0448000d04a880000
:10463800222120000200e600d24a8800f25520001c
:104648000280e600d24a8800d04a80000301200098
:104658000300b90043062000110009004308d800f0
:10466800a056880087f93700f0448000e04a8800a7
:10467800222120000200e600e24a8800f2552000cc
:104688000280e600e24a8800e04a80000301200038
:104698000300b90043062000110009004308d800b0
:1046a800b056880077f9370010458000f04a880036
:1046b800222120000200e600f24a8800f25520007c
:1046c8000280e600f24a8800f04a800003012000d8
:1046d8000300b90043062000110009004308d80070
:1046e800c056880067f9370030458000004b8800c5
:1046f800222120000200e600024b8800f25520002b
:104708000280e600024b8800004b80000301200075
:104718000300b90043062000110009004308d8002f
:10472800d056880057f9370030578000304c880041
:1047380040578000404c880052f93700505780009d
:10474800504c88004ff9370062a9aa004df937008c
:104758006269aa004bf937006249aa0049f9370093
:104768006289aa00000820006289ae0000002000cb
:104778008052880043f937009a29aa0041f9370086
:104788009a09aa00000820006289ae0000002000f3
:10479800805288003bf937004669a8006a43020046
:1047a8000000000037f937004689aa0035f93700bc
:1047b8006229aa0033f937006e89aa00a429ef00fc
:1047c8006e89ae003c49a9006e89ae003c69a9001b
:1047d8006e89ae00040037000400fc00e09324005a
:1047e8004009880027f937000400fc00f0ff270083
:1047f8004009880023f937003c09a8008029ec000b
:10480800f1012000004c80000180e6008029ed00c5
:104818001cf937003c09a8008029ed0019f93b0074
:104828008029ec0017f937004a2aec0081002000a3
:10483800505280000180e6004a2aef0011f9370043
:104848004a2aed000ff93b007300200053528800fc
:104858000cf937004c2aec00a100200060528000bf
:104868000180e6004c2aef0006f937004e2aec00da
:10487800b1002000705280000180e6004e2aef004f
:1048880000f937004c2aed00fef83b0093002000a9
:1048980063528800fbf837004e2aed00f9f83b0018
:1048a800a300200073528800f6f8370010458000f6
:1048b800604c8800030120000300b9004306200073
:1048c800110009004308d800e0568800edf83700c9
:1048d8003d29a80046c9a800d0448000704588003a
:1048e800f04480008045880010458000904588008d
:1048f80030458000a0458800e2f837000000060037
:10490800c0438000011020000100e6001c003700b1
:104918008000eb0079e8af008080eb00c0438000a6
:10492800000202000000000043da2300f2ff2f001b
:1049380056020200000000004629ae0004003700bd
:10494800fe03020000000000b043880000000600db
:10495800032024000200200042030200000000009f
:10496800e3f02300428e23005602020000000000fc
:10497800fe03020000000000b043880000000600ab
:104988008000eb007de8af008080eb00e043800012
:10499800000202000000000043da2300f2ff2f00ab
:1049a80056020200000000004629af00040037004c
:1049b800fe03020000000000b0438800000006006b
:1049c80063fe230062662600560202000000000013
:1049d800fe03020000000000020220000200400066
:1049e800b04388000000060000020200000000003a
:1049f80073f22300f2472300560202000000000071
:104a0800fe0302000000000000000600f401fc00a4
:104a18000002020000000000e3488000f248800025
:104a280042030200000000004c09e2000a003200c4
:104a3800654a800061836a000a00320062836a0066
:104a48000b00320063836a000c00320093142400c8
:104a580012f629000c0037006300240012a4260077
:104a680009003700930c240012f6290006003700cd
:104a78006310240012a426000300370073112400d9
:104a8800f2882900000037005602020000000000ea
:104a980001f0a600020037008000eb000000eb00e8
:104aa8000149880010498800fe0302000000000048
:104ab800a048880001f0a7001429ef000100e000d9
:104ac8000100320000000600120020000200e6008b
:104ad800000006000149800010498000937e2300f1
:104ae80042452000560202000000000001f0a70025
:104af8000600370023498000324980004403020041
:104b0800000000002149880030498800fe030200a7
:104b18000000000001f0a600b04888000000060070
:104b2800205b80000000ea008000eb0000f0a70096
:104b38008080eb000002020000000000831c2400bb
:104b480002002000be02020000000000835980001d
:104b5800925980005602020000000000fe03020085
:104b68000000000000428800a1f53700e0548000f2
:104b78008000eb0000f0a7008080eb00000202003c
:104b8800000000000302240002002000be02020010
:104b980000000000e3598000f2598000560202002c
:104ba80000000000fe030200000000002042880010
:104bb8000000060000428000c14280000001780029
:104bc8000180e600010178008100ea000100e600aa
:104bd800010178000242880000428000c141800043
:104be8003c26020000000000404280005142800044
:104bf8005042880052260200000000005826020099
:104c0800000000008626020000000000204280000c
:104c1800b1428000000178000180e60001017800bf
:104c28008100ea000100e6000101780022428800c4
:104c380020428000914180003c26020000000000d4
:104c48004042800061428000604288005226020093
:104c5800000000001827020000000000462702009c
:104c680000000000e04b8000c051880000000600f2
:104c7800010050008001780001802000020021001e
:104c88000180e600820150008100ea000100e60090
:104c980082014000434288000000060001005000e5
:104ca8007042880000000600404280000120200079
:104cb8000180e6005028ef000180e6001000370070
:104cc8008100ea000100e6005028ef000100e6003c
:104cd8000b00370040428000814280000100400004
:104ce80080017800027122000298e6000200780034
:104cf8000201ea000218e6000200780080428800fb
:104d080000000600404280008000eb0000f0a70091
:104d18008080eb000002020000000000832c2400c9
:104d280002002000be02020000000000635980005b
:104d38007259800056020200000000006155880088
:104d480070558800704280008000eb0000f0a700da
:104d58008080eb000002020000000000831c240099
:104d680002002000be02020000000000a3598000db
:104d7800b2598000560202000000000081558800e8
:104d880090558800804280008000eb0000f0a7006a
:104d98008080eb000002020000000000c3692400cc
:104da80002002400be02020000000000c359800077
:104db800d25980005602020000000000a155880068
:104dc800b055880063558000725580004403020086
:104dd80000000000835580009255800044030200c3
:104de800000000006e69af0001f0a200fe0302009f
:104df80000000000624b8000020040008001780043
:104e0800614b8000c10bb000624b8000c20bb10047
:104e18000180e600810178000200e6008201780046
:104e2800d351880000000600404280000120200085
:104e38000180e6005228ef000180e60010003700ec
:104e48008100ea000100e6005228ef000100e600b8
:104e58000b00370040428000914280000100400072
:104e680080017800027122000298e60002007800b2
:104e78000201ea000218e600020078009042880069
:104e880000000600404280008000eb0000f0a70010
:104e98008080eb000002020000000000832c240048
:104ea80002002000be0202000000000063598000da
:104eb800725980005602020000000000c1558800a7
:104ec800d0558800704280008000eb0000f0a700f9
:104ed8008080eb000002020000000000831c240018
:104ee80002002000be02020000000000035a8000f9
:104ef800125a80005602020000000000e1558800a6
:104f0800f0558800904280008000eb0000f0a70078
:104f18008080eb000002020000000000c36924004a
:104f280002002400be02020000000000235a800094
:104f3800225a800056020200000000000156880034
:104f480010568800c3558000d255800044030200e3
:104f580000000000e3558000f25580004403020081
:104f6800000000006e09af0001f0a200fe0302007d
:104f780000000000d24b8000020040008001780051
:104f8800d14b8000c10bb000d24b8000c20bb100e6
:104f98000180e600810178000200e60082017800c5
:104fa800a35188000000060080022000d141800043
:104fb8000088e6000d003700714180000088e60097
:104fc8000a003700a14180000088e600070037008a
:104fd8005448a9005468a9005428a9005408a900f5
:104fe80020002000404d8800000006005428a8003a
:104ff8005408a800414d80000160010002003700fc
:105008000e0037000d0037005448a8005468a80067
:1050180020002000314d80000100e700000006005c
:10502800000020000100e7005468a90010002000db
:105038000100e7005448a900000006005448a900f0
:105048005468a900000006003d69a9003d89a9002f
:10505800d0418000714d8000010050008000eb00bd
:1050680000f0a7008080eb000002020000000000b2
:10507800c3488000d2488000be0202000000000041
:10508800fe03020000000000f04188009123200088
:105098000180e600f141880071dc2f000100e60084
:1050a800f141880070418000514d8000010050009e
:1050b8008209af000000ea008000eb0000f0a700c2
:1050c8008080eb000002020000000000c34880005e
:1050d800d2488000be02020000000000fe03020069
:1050e8000000000090418800912320000180e60024
:1050f8009141880071dc2f000100e6009141880091
:10510800d0418000714d8000010050001400330030
:105118009041800001202000030020000300e600e9
:10512800070037000100e6002c003700f04180003e
:10513800014020000080500090418800270037007f
:105148008100ea000180e60024003700f041800079
:1051580001c02f0000804000904188001f003700e8
:105168009041800001202000030020000300e60099
:105178000c0037000100e600050037000140200060
:10518800f0418000008050009041880013003700f3
:1051980001802000904180000080500090418800ec
:1051a8000e0037009041800001e02f00030020002e
:1051b8000180e6000500370001c02f00f0418000a3
:1051c80000804000904188000400370001802f00d3
:1051d80090418000008050009041880090418000fc
:1051e800310720000180e600040037008100ea0052
:1051f8000100e600010037003d69a800a0418000d9
:10520800614d8000010050008229af000000ea00d3
:105218008000eb0000f0a7008080eb000002020095
:1052280000000000c3488000d2488000be0202008f
:1052380000000000fe03020000000000c0418800da
:10524800912320000180e600c141880071dc2f0015
:105258000100e600c1418800d0418000714d800006
:105268000100500014003300c041800001202000dc
:10527800030020000300e600070037000100e600f5
:105288002c003700f04180000140200000805000d1
:10529800c0418800270037008100ea000180e6004d
:1052a80024003700f041800001c02f00008040003a
:1052b800c04188001f003700c04180000120200045
:1052c800030020000300e6000c0037000100e600a0
:1052d8000500370001402000f041800000805000a8
:1052e800c04188001300370001802000c0418000c1
:1052f80000805000c04188000e003700c041800087
:1053080001e02f00030020000180e60005003700bf
:1053180001c02f00f041800000804000c04188009b
:105328000400370001802f00c04180000080500039
:10533800c0418800c0418000310720000180e6009c
:10534800000006008100ea000100e60000000600f7
:105358003d89a8005428ae0000000600d041800016
:10536800804d880000000600904180003300200036
:10537800110009000300d800010020000100e70027
:10538800060037000180e600020037000100210016
:1053980000804000010021000080500080588800f3
:1053a80090418000010020000100e700060037005e
:1053b8000180e60002003700010021000080400063
:1053c800010021000080500090588800c0418000f2
:1053d800010020000180e6000200370001002100e2
:1053e8000080400003012000110009000380d8005c
:1053f800a05888000000060010002000414d8000e1
:105408000180e7000000060010002000214d800008
:105418000180e700000006004449af0003003700a0
:105428005448a9005468a900000006005448a80080
:105438005468a800000006008000eb0021ebaf00d4
:105448008080eb000059800000020200000000008c
:105458008101780000017800560202000000000077
:10546800c15d8800d05d8800c15a8000d05a800094
:1054780000020200000000008101780000017800ad
:105488005602020000000000c35d8000d25d80006b
:1054980044030200000000007a040200000000003b
:1054a800fe03020000000000e15a8800f05a88005c
:1054b80000000600c15a8000d05a80000002020095
:1054c80000000000c15d8800d05d88008000eb000e
:1054d80021ebaf008080eb00005980000002020041
:1054e80000000000c35d8000d25d8000400402001f
:1054f800000000005326240012ee2200560202008b
:1055080000000000fe03020000000000505988005f
:10551800000006000ac8a9000ae8a9000b88a9002b
:10552800a6cf20000b68af00a6e02000b6027800e6
:10553800770420000728e7002600370067052000c9
:105548000728e70004003700270520000728e700a0
:105558004f00370090043700b60278004705200056
:1055680007a8e70000000600b602780077042000cc
:1055780007a8e7000000060046cf20000b68af0030
:1055880046e020009800200067000700e9c92000d5
:10559800980020006b000700480020006200070008
:1055a8009800200060000700480020005e00070007
:1055b800880020005c000700480020005a0007000f
:1055c800c9ca2000880020005e0007000ae8a80079
:1055d80000000600b60278007704200007a8e7005c
:1055e80000000600b60278001704200007a8e700ac
:1055f8000000060046cf20000b68af0046e0200000
:105608009800200048000700d80020004600070046
:1056180009c32000e80020004a00070089c42000d0
:105628004800200047000700c9c42000f8002000f7
:105638004400070069c62000480020004100070018
:10564800a9c62000480020003e000700e9c6200047
:10565800580020003b00070049c7200068002000d0
:1056680038000700e9c7200098002000350007002f
:10567800e9c8200098002000320007000ac8a800e6
:105688000a28ae00000006000a28a900000006004b
:10569800b6027800d704200007a8e700000006003b
:1056a800b60278003704200007a8e70000000600cb
:1056b80046cf20000b68af0046e02000980020008d
:1056c80019000700d80020001700070049ce200065
:1056d800480020001b000700b80020001200070047
:1056e8004800200010000700c80020000e00070036
:1056f800480020000c000700980020000a0007005e
:10570800a80020000800070069ce200088002000bb
:105718000c0007000b88a8000a28ae00000006004d
:105728000a28a900000006000804e9001a0432004b
:10573800b6027800c702200007a8e700faff370082
:10574800000006000804e90013043200b6027800dd
:10575800851c7800c702200007a8e700f9ff37007a
:1057680000000600b8f1070066ce200009c120003d
:1057780060cf200030618800442c02000000000047
:105788000ba8af00000006002060800010588800b9
:10579800106080002058880000000600aaf1070069
:1057a80046c7200009c1200020c8200030618800b9
:1057b800ea2b0200000000001060800030588800ca
:1057c8005058800040588800000006000bc8a90007
:1057d8000a2bef000004eb00242cef000e0ca900ac
:1057e800242cec008002eb00b6027800c7022000ef
:1057f8000728e70015003700e70220000728e70020
:105808000f003700376180000638e60018003700bf
:10581800d70220000728e70006003700f70020001d
:1058280087836200871c78000bc8af000804e80073
:10583800ebff37000e0ca800242ced00e8ff370022
:105848000bc8a800242ced00e5ff3700242ced0040
:1058580058588800240ce20005003200240ced00a2
:10586800a80e0200000000000ba8a9000000060016
:10587800022cef00042cef000ba8a8000000060083
:10588800242cef000e0ca900242cec00b6027800a2
:10589800c70220000728e70010003700e7022000b1
:1058a8000728e7000d003700376180000638e6005a
:1058b80012003700d70220000728e700040037004d
:1058c800f700200087836200871c7800eeff37000e
:1058d8000e0ca800242ced00ebff3700242ced0063
:1058e800240ce20005003200240ced00a80e020092
:1058f800000000000ba8a90000000600022cef0021
:10590800042cef000ba8a800000006004ef10700c9
:10591800e6c6200009c1200040c720003061880089
:10592800242cef00242cec00b6027800f7002000ad
:1059380087836200871c7800c70220000728e700d9
:1059480004003700376180000638e60001003700a0
:10595800f4ff37008024eb00242ced000000370012
:10596800240ce2008c033200240ced00a80e020087
:105978000000000010608000905a8800280f020084
:105988000000000056638000f50020000503630056
:105998008660880000002000a80e020000000000b9
:1059a80010608000a05a88000000060026f1070059
:1059b800c6ca200009c12000e0cb20003061880061
:1059c800ea2b0200000000002160800010608000c7
:1059d8004629af0017003700555880000500e00041
:1059e8001200320061836a000d00320062836a008f
:1059f8000700320063836a00010032002a00370082
:105a0800833e2000110009004308d8000700370032
:105a180043062000110009004308d800030037009e
:105a2800a3002000110009004308d800805a88000c
:105a38000000060000020200000000005558800027
:105a48000500e0001000320061836a000b0032009c
:105a580062836a000600320063836a000100320034
:105a680011003700834c2400020020000800370092
:105a78000332240002002000050037000318240028
:105a88000200200002003700c3fc2300d2cc2c0007
:105a9800be02020000000000fe0302000000000039
:105aa800805a880000000600502bef000000060016
:105ab800e5f00700e6c9200009c1200000cb20005e
:105ac80030618800ea2b020000000000216080009d
:105ad800106080000002020000000000555880009d
:105ae8000500e0000f00320061836a000b003200fd
:105af80062836a000600320063836a000100320094
:105b080071003700a3472400020020000500370079
:105b1800832c240002002000020037000312240016
:105b280002002000be02020000000000c15e8800e2
:105b3800d05e8800fe03020000000000c058880004
:105b4800c15e8000d05e800063f3230012b620009f
:105b58005602020000000000c15e8800d05e880086
:105b6800fe03020000000000b05888000000060094
:105b7800b5f00700e6c8200009c1200000ca2000cf
:105b880030618800ea2b02000000000021608000dc
:105b980010608000704e880000000600aaf0070020
:105ba800e6c7200009c1200000c920003061880034
:105bb800ea2b0200000000002160800010608000d5
:105bc800604e880000020200000000005558800066
:105bd8000500e0001000320061836a000b0032000b
:105be80062836a000600320063836a0001003200a3
:105bf8003500370073b52300c23520000800370090
:105c080063d02300a22126000500370073ea230091
:105c180002aa2f00020037001305240082942f00e7
:105c28005602020000000000d1588800e0588800a1
:105c3800135980002259800042030200000000002e
:105c48004629af0004003700c3e92300f2eb200027
:105c580056020200000000004149880050498800af
:105c6800fe0302000000000000598800414980003e
:105c780050498000335980004259800031598800ca
:105c880040598800420302000000000083242400d9
:105c9800020020005602020000000000814988002e
:105ca80090498800fe03020000000000005b8800a5
:105cb800d1588000e0588000fe0302000000000078
:105cc800f058880000000600000006000a68a800d6
:105cd80000000600242cef00242cec00b60278000b
:105ce800f700200087836200871c7800e702200005
:105cf8000728e70007003700c70220000728e70049
:105d080004003700376180000638e60001003700dc
:105d1800f1ff37008024eb00242ced000000060082
:105d28000a88a9000e0ca900242cef00242cec00f2
:105d3800b6027800f700200087836200871c78008d
:105d4800e70220000728e7000a003700d7022000f2
:105d58000728e7000a000700c70220000728e70015
:105d68000b003700376180000638e6000100370075
:105d7800eeff37008024eb00242ced000000060025
:105d88000e0ca800242ced00a902780000000600e3
:105d98000a88a80000000600242cec00b60278004f
:105da800f700200087836200871c7800c702200064
:105db8000728e70004003700376180000638e6004e
:105dc80001003700f4ff37008024eb00242ced009d
:105dd800000006001cf0070009c320003903780002
:105de800f500200005036300866088003903780009
:105df800f5002000050363009660880039037800e9
:105e0800f500200005036300a660880039037800c8
:105e1800f500200005036300b660880039037800a8
:105e280088c120000300080003000000390378003f
:105e3800f500200005036300061c78000e0ca9007d
:105e480046628000350520000628e7000e0ca800f1
:105e580070002000a80e02000000000020608000f2
:105e6800706688001060800060668800f6ef0700a2
:105e7800c9c4200039037800f50020000503630039
:105e88008660880039037800f50020000503630068
:105e98009660880039037800f50020000503630048
:105ea800a660880039037800f50020000503630028
:105eb800b660880039037800f50020000503630008
:105ec800c660880039037800a8c1200003000800d4
:105ed8000300000039037800f50020000503630083
:105ee800061c78000e0ca9003663800055042000bb
:105ef8000628e7000e0ca80080002000a80e02006b
:105f0800000000002060800090668800106080001b
:105f18008066880000000600cbef070086618000dd
:105f2800f500200005036300866088009661800004
:105f3800f500200005036300966088000e0ca90098
:105f480010002000a80e0200000000002160800060
:105f5800106080000002020000000000f165880067
:105f6800e0658800b8ef070049c3200039037800ce
:105f7800f500200005036300866088003903780077
:105f8800f500200005036300966088003903780057
:105f980048c120000500080003000000390378000c
:105fa800f500200005036300061c78000e0ca9000c
:105fb80070002000a80e0200000000002160800090
:105fc80010608000000202000000000043c62400a8
:105fd800021c2e00be02020000000000f3658000d3
:105fe800e26580004403020000000000e3c82300cb
:105ff80052a32f00560202000000000001f0a0008a
:1060080046628000e50420000628e70001f0a100b0
:1060180031668800206688008bef07006662800082
:10602800f500200005036300866088007662800022
:10603800f5002000050363009660880086628000f2
:10604800f500200005036300a66088000e0ca90077
:1060580020002000a80e020000000000216080003f
:10606800106080000002020000000000f165880056
:10607800e065880074ef070029c52000390378001f
:10608800f500200005036300866088003903780066
:10609800f500200005036300966088003903780046
:1060a80048c12000050008000300000039037800fb
:1060b800f500200005036300061c78000e0ca900fb
:1060c80070002000a80e020000000000216080007f
:1060d80010608000000202000000000043c6240097
:1060e800021c2e00be02020000000000f3658000c2
:1060f800e26580004403020000000000e3c82300ba
:1061080052a32f00560202000000000001f0a00078
:1061180036638000750520000628e70001f0a1001d
:10612800516688004066880000000600a05a80007a
:10613800010020000100e60000000600905a8000df
:10614800310020000100e60000000600da300200fd
:1061580000000000f0568000a14a80000100e6001f
:106168000000060050668000505f8800406680008e
:10617800405f880030668000305f880020668000bd
:10618800205f8800d058800010598800e0588000af
:1061980020598800fa2aef00f82aef00f62aef00c3
:1061a8004609a8000b08a80000000600060be2003c
:1061b80001003a000600370030588000b14a8000dc
:1061c8000180e60002003700de2aec00000006002d
:1061d800de2aef000000060031668000206680009d
:1061e800c3528000b2528000420302000000000047
:1061f800e404020000000000030024000001eb009a
:10620800be02020000000000810178000001780051
:106218005602020000000000815d8800905d880041
:106228003166800020668000e8040200000000005b
:10623800c15d8800d05d8800a15d8800b05d8800e0
:10624800c1528000b0528000e80402000000000043
:10625800a35d8000b25d80005602020000000000cd
:10626800a15d8800b05d88005166800040668000ae
:10627800e3528000d2528000420302000000000076
:10628800e404020000000000030024000001eb0009
:10629800be020200000000008101780000017800c1
:1062a8005602020000000000a35d8000b25d80007d
:1062b8005602020000000000835d8000925d8000ad
:1062c80044030200000000007a04020000000000fd
:1062d800ec04020000000000030024000001eb00b1
:1062e8005602020000000000815d8800905d880071
:1062f8004629af000300370023ac240062be240007
:1063080002003700f3b9240092d225005602020099
:1063180000000000fe030200000000009152880007
:10632800a0528800815d8000905d8000e404020036
:1063380000000000c35d8000d25d800056020200ac
:1063480000000000a15d8800b05d8800815d8000cc
:10635800905d8000e804020000000000815d880074
:10636800905d88003166800020668000e4040200a9
:1063780000000000835d8000925d800056020200ec
:1063880000000000815d8800905d8800c152800097
:10639800b0528000e404020000000000835d800029
:1063a800925d80004203020000000000a35d8000af
:1063b800b25d8000be02020000000000815d88001e
:1063c800905d880003f823000001eb0044030200fd
:1063d80000000000835d8000925d800001f0a6004f
:1063e8000200370003f82b000001eb00830078005f
:1063f80002007800f004020000000000815d8800bf
:10640800905d8800e1528000d05280005366800081
:10641800426680004203020000000000e40402001b
:106428000000000001f0a6000b003700815d80002d
:10643800905d80002322240032982f00560202002b
:1064480000000000e15d8800f05d8800fe030200a6
:106458000000000010003700910c2400b0fd20005f
:10646800835d8000925d800042030200000000000e
:10647800815d8800905d88002322240032982f00d7
:106488005602020000000000e15d8800f05d88000f
:10649800fe03020000000000b25880000200500015
:1064a8000110200000f0a6008000eb000100400071
:1064b8008052880000000600316680002066800057
:1064c800335f8000225f800042030200000000006a
:1064d800e404020000000000030024000001eb00b7
:1064e800be0202000000000081017800000178006f
:1064f8005602020000000000815d8800905d88005f
:106508003166800020668000e80402000000000078
:10651800c15d8800d05d8800a15d8800b05d8800fd
:10652800315f8000205f8000e80402000000000066
:10653800a35d8000b25d80005602020000000000ea
:10654800a15d8800b05d88005166800040668000cb
:10655800535f8000425f8000420302000000000099
:10656800e404020000000000030024000001eb0026
:10657800be020200000000008101780000017800de
:106588005602020000000000a35d8000b25d80009a
:106598005602020000000000835d8000925d8000ca
:1065a80044030200000000007a040200000000001a
:1065b800ec04020000000000030024000001eb00ce
:1065c8005602020000000000815d8800905d88008e
:1065d8004629af000300370023ac240062be240024
:1065e80002003700f3b9240092d2250056020200b7
:1065f80000000000fe03020000000000c15a8800ed
:10660800d05a8800815d8000905d8000e40402001b
:1066180000000000c35d8000d25d800056020200c9
:1066280000000000a15d8800b05d8800815d8000e9
:10663800905d8000e804020000000000815d880091
:10664800905d88003166800020668000e4040200c6
:1066580000000000835d8000925d80005602020009
:1066680000000000815d8800905d8800315f800037
:10667800205f8000e404020000000000835d8000c9
:10668800925d80004203020000000000a35d8000cc
:10669800b25d8000be02020000000000815d88003b
:1066a800905d880003f823000001eb00440302001a
:1066b80000000000835d8000925d800001f0a6006c
:1066c8000200370003f82b000001eb00830078007c
:1066d80002007800f004020000000000815d8800dc
:1066e800905d8800515f8000405f800053668000a5
:1066f800426680004203020000000000e404020039
:106708000000000001f0a6000b003700815d80004a
:10671800905d80002322240032982f005602020048
:1067280000000000515a8800605a8800fe030200e9
:106738000000000010003700910c2400b0fd20007c
:10674800835d8000925d800042030200000000002b
:10675800815d8800905d88002322240032982f00f4
:106768005602020000000000515a8800605a880052
:10677800fe03020000000000b25880000200500032
:106788000110200000f0a6008000eb00010040008e
:10679800405a8800000006000000060031668000ac
:1067a80020668000a3c52400920e2900560202002c
:1067b80000000000fe03020000000000b16688002f
:1067c800a06688005166800040668000a3c524004a
:1067d800920e29005602020000000000fe0302008b
:1067e80000000000d1668800c0668800515f800004
:1067f800405f8000a3c52400920e290056020200c3
:1068080000000000fe03020000000000915f880005
:10681800805f8800315f8000205f8000a3c524006e
:10682800920e29005602020000000000fe0302003a
:1068380000000000715f8800605f880000000600ab
:10684800e4458800f5458800064688000b68ae00d8
:106858001e0037005461800045cf20000428e7005f
:1068680013003700b5118000051a780054618800bc
:10687800a600200006a8e700070037000b48a8007c
:106888000b68aa0044cf20000b68ae0044e020004b
:10689800546188002b00370086da200004b0e60037
:1068a8002800370044cf20005461880025003700b5
:1068b800b51180004602200006a8e7002100370035
:1068c800051a7800546188001e0037005461800062
:1068d80045e020000428e70013003700b5118000c8
:1068e800051a780054618800a600200006a8e70071
:1068f800070037000b48a8000b68aa0044cf200007
:106908000b68ae0044e02000546188000d00370099
:1069180086eb200004b0e6000a00370044e02000bf
:106928005461880007003700b51180004602200036
:1069380006a8e70003003700051a780054618800ac
:10694800000037003202af00c0ff3700e445800086
:10695800f5458000064680003222a90087c0a900bc
:10696800004006008460a9000040060000a0fe0068
:10697800849fbe00869fbe00889fbe008a9fbe007f
:106988008c9fbe00bb0180002b5e8800cb0180007d
:106998003b5e8800db0180004b5e8800eb018000d5
:1069a8005b5e8800fb0180006b5e88000b02800044
:1069b8007b5e88000060fe004449af00020037009b
:1069c80084e0a90094e0a8000b28aa000b28af00d7
:1069d80001003700cf003700c2110200000000009c
:1069e800f42aec00aa5780004b0620000bd0e700e1
:1069f80074003700f42aef00f62aec00ba5780003a
:106a0800cb0320000bd0e70008003700f62aef0080
:106a1800f82aec00ca578000cb0320000bd0e7000f
:106a280002003700f82aef00fa2aec000b08af0042
:106a380064003700fa0ae20062003a00f80ae2004d
:106a480060003a003a002000bb5780000b50e70076
:106a58004a0037004a002000bb5780000b50e7006f
:106a6800440037005a002000bb5780000b50e70055
:106a7800200037006a002000bb5780000b50e70059
:106a88002c0037007a002000bb5780000bd0e700ad
:106a98004c0037004449af000c48a8004449a900fd
:106aa8000c48ae00470037008420a9009420a900b4
:106ab80084a0a90094a0a90088a0a90098a0a90072
:106ac80088c0a90098c0a90088e0a90098e0a9009a
:106ad8008440a9009440a90084c0a90094c0a900da
:106ae8008720a9009720a9008740a9009740a900fe
:106af800340037003342a8000100200091018800cb
:106b0800c147240033000800060000000000eb0025
:106b18003140ba003302ae00feff37000a00090018
:106b280000000000a01188003302ae00feff37000d
:106b38009c0037003342a800010020009101880022
:106b4800414c240011000800060000000000eb0082
:106b58003140ba003302ae00feff37000a000900d8
:106b680000000000a01188003302ae00feff3700cd
:106b78008c00370000042000c01188003342a800b0
:106b88000100200091018800014b24001300080037
:106b9800060000000000eb003140ba003302ae00ee
:106ba800feff37000a00090000000000a01188005d
:106bb8003302ae00feff3700a0022000c01188009b
:106bc800780037000b08af0023003700fa0ae2000c
:106bd80021003a00f80ae2001f003a008200200073
:106be800b35780000218e6002a003700c2012000cf
:106bf800b35780000298e600170037008000eb00ca
:106c0800904880000002020000000000014988004e
:106c180010498800e1488000f0488000833424004f
:106c28000200200056020200000000000349800014
:106c3800124980004403020000000000933424003d
:106c480002002000be02020000000000e1488800a7
:106c5800f04888000f003700f21202000000000020
:106c68008000eb009048800068f70700d8270200f2
:106c7800000000005408ae00060037002828020073
:106c880000000000b829020000000000de25020014
:106c98000000000010418000110020000180e70082
:106ca800020037009a09af004bfd07001041800031
:106cb800210020000180e700020037000b08af0028
:106cc800fdfd070010418000310020000180e70031
:106cd80005003700204d8000110020000180e600eb
:106ce8004c0f02000000000010418000410020000d
:106cf8000180e70002003700002a020000000000bf
:106d080010418000510020000100e6002228ec001c
:106d1800240037000ae8ae000f0037003e29ef00d4
:106d280022fb070062fb07009cfe07008000eb00c7
:106d3800504880002cf70700704888008000eb005e
:106d48006048800028f707008048880084240200f3
:106d5800000000000ae8a9000ac8ae000a003700cf
:106d68002228ef00d22b020000000000e7fa0700fb
:106d780069fc070089fb07007dfb07000b08ae00d4
:106d8800eafc07000ac8a9000b88ae000500370016
:106d98003e29ef0073fa0700a7f90700c5f90700b5
:106da8000b88a900d442020000000000b6130200bc
:106db8000000000078150200000000002e420200ca
:106dc8000000000040418000234d80003200200078
:106dd8000218e7000059880030418000234d8000e8
:106de800320020000218e700405a88000b48af0024
:106df8008e2a0200000000000b48a9004b5e8000ac
:106e0800db0188005b5e8000eb0188006b5e800020
:106e1800fb0188007b5e80000b0288008400a900cb
:106e28008780a9004f06be004f05be004f04be0074
:106e38004f03be004f02be000080fe000040060067
:106e48009780a90097c0a900c0458800d14588004f
:106e58002342a8000a00fc0080408000a104200012
:106e68000180e6004e003700000078004c00330037
:106e7800006001004a003700520037005a0037000e
:106e88006700370074003700810037008e00370034
:106e98009b003700a8003700b5003700c200370054
:106ea800cf003700dc003700e9003700f600370074
:106eb80003013700100137001d0137002a01370090
:106ec8003701370044013700510137005e013700b0
:106ed8006b013700780137008501370092013700d0
:106ee8009f013700ac013700b9013700c6013700f0
:106ef800d3013700db013700e3013700eb0137002e
:106f0800f3013700fb013700030237001002370096
:106f18001d0237002a023700370237003e023700c9
:106f28004b023700580237006502370072023700fb
:106f38007f0237008c02370099023700a60237001b
:106f4800b3023700c0023700cd023700da0237003b
:106f5800e7023700f4023700010337000e03370059
:106f68001a03370026033700320337003e03370081
:106f78004a03370056033700620337006e033700b1
:106f88007a03370086033700920337009e033700e1
:106f9800aa033700b6033700c2033700ce03370011
:106fa8008040800020118800b057800020118800a0
:106fb800c057800020118800d05780002011880019
:106fc800c503370080408000201188007058800079
:106fd80020118800a058800020118800b058800037
:106fe80020118800bc0337008040800020118800f1
:106ff80000598000f10f20000080600020118800f7
:107008000059800001f02f00008060000080fd0022
:10701800201188003043800020118800ae0337001b
:107028008040800020118800c0668000f10f200099
:107038000080600020118800c066800001f02f00e9
:10704800008060000080fd0020118800b05a800098
:1070580020118800a003370080408000201188009c
:10706800d0668000f10f20000080600020118800a9
:10707800d066800001f02f00008060000080fd00d5
:1070880020118800905a8000201188009203370050
:107098008040800020118800a0668000f10f200049
:1070a8000080600020118800a066800001f02f0099
:1070b800008060000080fd0020118800a05a800038
:1070c8002011880084033700804080002011880048
:1070d800b0668000f10f2000008060002011880059
:1070e800b066800001f02f00008060000080fd0085
:1070f80020118800405a800020118800760337004c
:107108008040800020118800605f8000f10f20001f
:107118000080600020118800605f800001f02f006f
:10712800008060000080fd0020118800304a800047
:1071380020118800680337008040800020118800f3
:10714800705f8000f10f200000806000201188002f
:10715800705f800001f02f00008060000080fd005b
:1071680020118800f0568000201188005a0337004b
:107178008040800020118800805f8000f10f20008f
:107188000080600020118800805f800001f02f00df
:10719800008060000080fd0020118800204b8000e6
:1071a800201188004c03370080408000201188009f
:1071b800905f8000f10f200000806000201188009f
:1071c800905f800001f02f00008060000080fd00cb
:1071d8002011880010438000201188003e033700ea
:1071e800804080002011880070488000f10f200046
:1071f80000806000201188007048800001f02f0096
:10720800008060000080fd0020118800204380007d
:10721800201188003003370080408000201188004a
:10722800d05a8000f10f20000080600020118800f3
:10723800d05a800001f02f00008060000080fd001f
:1072480020118800304b800020118800220337006d
:107258008040800020118800805a8000f10f2000b3
:107268000080600020118800805a800001f02f0003
:10727800008060000080fd0020118800404b8000e5
:1072880020118800140337008040800020118800f6
:10729800c0588000f10f2000008060002011880095
:1072a800c058800001f02f00008060000080fd00c1
:1072b80020118800104b8000201188000603370039
:1072c8008040800020118800a0488000f10f200035
:1072d8000080600020118800a048800001f02f0085
:1072e800008060000080fd0020118800705680003a
:1072f80020118800f80237008040800020118800a3
:1073080080488000f10f2000008060002011880074
:107318008048800001f02f00008060000080fd00a0
:10732800201188009056800020118800ea0237005a
:10733800804080002011880020588000f10f200034
:1073480000806000201188002058800001f02f0084
:10735800008060000080fd002011880080568000b9
:1073680020118800dc02370080408000201188004e
:1073780010588000f10f2000008060002011880064
:107388001058800001f02f00008060000080fd0090
:10739800201188006056800020118800ce02370036
:1073a800804080002011880030588000f10f2000b4
:1073b80000806000201188003058800001f02f0004
:1073c800008060000080fd00201188004058800087
:1073d80020118800c00237008040800020118800fa
:1073e80090438000f10f2000008060002011880089
:1073f8009043800001f02f00008060000080fd00b5
:1074080020118800604a800020118800b2023700ed
:107418008040800020118800b0488000f10f2000d3
:107428000080600020118800b048800001f02f0023
:10743800008060000080fd0020118800904a8000d4
:1074480020118800a40237008040800020118800a5
:10745800c05a8000f10f20000080600020118800d1
:10746800c05a800001f02f00008060000080fd00fd
:1074780020118800804a8000201188009602370079
:107488008040800020118800e05a8000f10f200021
:107498000080600020118800e05a800001f02f0071
:1074a800008060000080fd0020118800504a8000a4
:1074b8002011880088023700804080002011880051
:1074c800f05a8000f10f2000008060002011880031
:1074d800f05a800001f02f00008060000080fd005d
:1074e80020118800704a8000201188007a02370035
:1074f800804080002011880050598000f10f200042
:1075080000806000201188005059800001f02f0091
:10751800008060000080fd0020118800a04a8000e3
:10752800201188006c0237008040800020118800fc
:10753800b04a8000f10f2000008060002011880010
:10754800b04a800001f02f00008060000080fd003c
:1075580020118800404a8000201188005e02370010
:107568008040800020118800005b8000f10f20001f
:107578000080600020118800005b800001f02f006f
:10758800008060000080fd0020118800204a8000f3
:1075980020118800500237008040800020118800a8
:1075a80020488000f10f2000008060002011880032
:1075b8002048800001f02f00008060000080fd005e
:1075c80020118800504b80002011880042023700ab
:1075d800804080002011880030488000f10f200092
:1075e80000806000201188003048800001f02f00e2
:1075f800008060000080fd0020118800704b800032
:107608002011880034023700804080002011880053
:1076180040488000f10f20000080600020118800a1
:107628004048800001f02f00008060000080fd00cd
:1076380020118800904b8000201188002602370016
:107648008040800020118800a04b80002011880015
:10765800b04b800020118800c04b800020118800aa
:107668001d0237008040800020118800a05680004d
:1076780020118800b056800020118800c056800074
:1076880020118800140237008040800020118800f3
:10769800d056800020118800804b8000201188007f
:1076a800004c8000201188000b02370080408000c9
:1076b80020118800e049800020118800104c8000cb
:1076c80020118800204c8000201188000202370019
:1076d80080408000201188008044800020118800ac
:1076e8009044800020118800b04480002011880058
:1076f800f90137008040800020118800a0448000f4
:1077080020118800e056800020118800704c80000d
:1077180020118800f0013700804080002011880087
:10772800b0438000f10f2000008060002011880025
:10773800b043800001f02f00008060000080fd0051
:1077480020118800804c800020118800e201370059
:10775800804080002011880000448000f10f200044
:1077680000806000201188000044800001f02f0094
:10777800008060000080fd0020118800904c80008f
:1077880020118800d4013700804080002011880033
:1077980010448000f10f2000008060002011880054
:1077a8001044800001f02f00008060000080fd0080
:1077b80020118800a04c800020118800c6013700e5
:1077c800804080002011880020448000f10f2000b4
:1077d80000806000201188002044800001f02f0004
:1077e800008060000080fd0020118800b04c8000ff
:1077f80020118800b80137008040800020118800df
:10780800c04c800020118800505280002011880050
:1078180020118800b00137008040800020118800c6
:10782800e04c8000f10f20000080600020118800eb
:10783800e04c800001f02f00008060000080fd0017
:10784800201188006052800020118800a2013700b2
:107858008040800020118800f04c8000f10f20004b
:107868000080600020118800f04c800001f02f009b
:10787800008060000080fd002011880070528000a8
:107888002011880094013700804080002011880072
:10789800004d8000f10f200000806000201188005a
:1078a800004d800001f02f00008060000080fd0086
:1078b80020118800a0578000201188008601370019
:1078c8008040800020118800104d8000f10f2000ba
:1078d8000080600020118800104d800001f02f000a
:1078e800008060000080fd0020118800d04c8000de
:1078f800201188007801370080408000201188001e
:1079080090528000f10f2000008060002011880054
:107918009052800001f02f00008060000080fd0080
:107928002011880080528000201188006a013700e9
:107938008040800020118800a0528000f10f2000b4
:107948000080600020118800a052800001f02f0004
:10795800008060000080fd0020118800204d80001c
:10796800201188005c0137008040800020118800c9
:10797800805c8000f10f20000080600020118800ea
:10798800805c800001f02f00008060000080fd0016
:107998002011880060418000201188004e013700c6
:1079a8008040800020118800905c8000f10f20004a
:1079b8000080600020118800905c800001f02f009a
:1079c800008060000080fd00201188008041800058
:1079d8002011880040013700804080002011880075
:1079e800a05c8000f10f200000806000201188005a
:1079f800a05c800001f02f00008060000080fd0086
:107a080020118800b0418000201188003201370021
:107a18008040800020118800b05c8000f10f2000b9
:107a28000080600020118800b05c800001f02f0009
:107a3800008060000080fd0020118800e041800087
:107a48002011880024013700804080002011880020
:107a580080588000f10f200000806000201188000d
:107a68008058800001f02f00008060000080fd0039
:107a780020118800a04280002011880016013700dc
:107a88008040800020118800604e8000f10f2000a7
:107a98000080600020118800604e800001f02f00f7
:107aa800008060000080fd0020118800304d8000bb
:107ab80020118800080137008040800020118800cc
:107ac800704e8000f10f20000080600020118800b7
:107ad800704e800001f02f00008060000080fd00e3
:107ae80020118800404d800020118800fa003700de
:107af8008040800020118800804e8000f10f200017
:107b08000080600020118800804e800001f02f0066
:107b1800008060000080fd0020118800b04d8000ca
:107b280020118800ec003700804080002011880078
:107b3800904e8000f10f2000008060002011880026
:107b4800904e800001f02f00008060000080fd0052
:107b580020118800904d800020118800de00370039
:107b68008040800020118800a04e8000f10f200086
:107b78000080600020118800a04e800001f02f00d6
:107b8800008060000080fd0020118800a04d80006a
:107b980020118800d0003700804080002011880024
:107ba800a0418000f10f20000080600020118800b3
:107bb800a041800001f02f00008060000080fd00df
:107bc8002011880020118800c30037008040800001
:107bd8002011880070418000f10f200000806000b3
:107be800201188007041800001f02f0000806000a3
:107bf8000080fd002011880020118800b6003700a1
:107c08008040800020118800d0418000f10f2000c2
:107c18000080600020118800d041800001f02f0012
:107c2800008060000080fd0020118800201188007d
:107c3800a9003700804080002011880090588000fb
:107c4800f10f20000080600020118800905880000b
:107c580001f02f00008060000080fd0020118800e6
:107c6800201188009c003700804080002011880087
:107c7800f0588000f10f200000806000201188007b
:107c8800f058800001f02f00008060000080fd00a7
:107c980020118800201188008f0037008040800064
:107ca80020118800004f8000f10f20000080600044
:107cb80020118800004f800001f02f000080600034
:107cc8000080fd0020118800201188008200370004
:107cd8008040800020118800104f8000f10f2000a4
:107ce8000080600020118800104f800001f02f00f4
:107cf800008060000080fd002011880020118800ad
:107d0800750037008040800020118800204f8000d7
:107d1800f10f20000080600020118800204f8000b3
:107d280001f02f00008060000080fd002011880015
:107d380020118800680037008040800020118800ea
:107d4800304f8000f10f2000008060002011880073
:107d5800304f800001f02f00008060000080fd009f
:107d680020118800201188005b00370080408000c7
:107d780020118800404f8000f10f20000080600033
:107d880020118800404f800001f02f000080600023
:107d98000080fd0020118800201188004e00370067
:107da8008040800020118800504f8000f10f200093
:107db8000080600020118800504f800001f02f00e3
:107dc800008060000080fd002011880020118800dc
:107dd800410037008040800020118800604f8000fb
:107de800f10f20000080600020118800604f8000a3
:107df80001f02f00008060000080fd002011880045
:107e0800201188003400370080408000201188004d
:107e1800704f8000f10f2000008060002011880062
:107e2800704f800001f02f00008060000080fd008e
:107e3800201188002011880027003700804080002a
:107e480020118800804f8000f10f20000080600022
:107e580020118800804f800001f02f000080600012
:107e68000080fd0020118800201188001a003700ca
:107e78008040800020118800904f8000f10f200082
:107e88000080600020118800904f800001f02f00d2
:107e9800008060000080fd0020118800201188000b
:107ea8000d0037008040800020118800a04f80001e
:107eb800f10f20000080600020118800a04f800092
:107ec80001f02f00008060000080fd002011880074
:107ed80020118800000037001028ec008140800045
:107ee800a00420000088e6001028ef00c0458000ac
:107ef800d145800097c0a8008400a9009780a800f9
:107f080000400600d7468800e8468800f946880001
:107f1800d502af0010003700070a8000e84480004f
:107f28000838e6000300370088835300d7448800e8
:107f380004003700490d23000884540087034400d7
:107f4800d7448800d7468000e8468000f94680007c
:107f58008420a90000400600070a80004261af00a3
:107f6800fdff3700e7448800d7468000e8468000d8
:107f7800f94680008420a9000040060017478800c1
:107f88002847880039478800d522af0010003700fd
:107f9800270a8000084580000838e60003003700fb
:107fa80088835300f744880004003700490d2300f4
:107fb8000884540087034400f7448800174780006a
:107fc800284780003947800084a0a90000400600a7
:107fd800270a80004661af00fdff3700074588008b
:107fe80017478000284780003947800084a0a900ef
:107ff800004006005747880068478800794788008e
:10800800d542af0020003700470a8000284580008d
:108018000838e6000b0037008883530017458800ae
:108028006e89ae00130037004449a900684c8000ef
:1080380008b8e6004449a8000c48af004449a90024
:108048000c003700490d23000884540087034400be
:10805800174588006e89ae00060037004449a9001c
:10806800684c800008b8e6004449a8000c48af00f6
:108078004449a90057478000684780007947800035
:1080880088a0a90000400600470a80004a61af00a6
:10809800fdff370027458800574780006847800064
:1080a8007947800088a0a90000400600874788001b
:1080b80098478800a9478800d562af0010003700ac
:1080c800670a8000484580000838e600030037004a
:1080d800888353003745880004003700490d230082
:1080e8000884540087034400374588008747800088
:1080f80098478000a947800088c0a9000040060072
:10810800670a80004e61af00fdff370047458800d1
:108118008747800098478000a947800088c0a90049
:1081280000400600b7478800c8478800d94788003c
:10813800d482af002e003700870a8000684580008f
:108148000838e60003003700888353005745880045
:1081580004003700490d23000884540087034400b5
:10816800574588003821200008b8e6000600370087
:108178006e89ae004449a8000c48af004449a900e4
:108188004029ef0015003700f85520000838e600b0
:10819800060037006e89ae004449a8000c48af00bd
:1081a8004449a9004029ef000c0037004029ec00a1
:1081b800084a8000a70020006e89af00020037003f
:1081c80007c0e6004449a90007c0e6004029ef00bf
:1081d8000c48af004449a9002221ef00b7478000ae
:1081e800c8478000d947800088e0a9000040060001
:1081f800870a80005261af00fdff3700674588009d
:10820800b7478000c8478000d947800088e0a900a8
:10821800004006001746880028468800394688002e
:108228000c08af000b0037000be8a9000c08a800e9
:108238006e28ef007028ef005641a9005621a800cb
:108248005601a800a70a80005661af00f1ff370069
:1082580039003700a70a8000480d230008b8e60057
:1082680027003700c8ce220008b8e6002c003700e7
:108278000be8ae0022003700c851220008b8e6001b
:108288001f0037004813220008b8e6001300370023
:108298004896210008b8e60019003700c8572100a1
:1082a8000838e600160037007028ec006e28d70062
:1082b8006f68a900c80020008943800009c0e70052
:1082c8001b00370078438000984388002fe1a800fe
:1082d8009900a9000c28a800090037007028ec00b4
:1082e8006e28d7006f68a800c80020008943800066
:1082f80009c0e7000e0037007843800098438800e3
:108308000c08a9000be8a9006e28ef007028ef0000
:108318005641a9005621a8005601a90006003700b9
:108328000c08a8000be8a8006e28ef007028ef00e2
:108338005661af00b7ff370013e1a9008500a90017
:108348000a21ef0013e1a8001746800028468000a4
:10835800394680008900a90000400600c44688000c
:1083680024002000540c8800c44680008440a900e2
:10837800004006000447880024002000840c880080
:108388000447800084c0a9000040060044478800d4
:1083980024002000b40c8800444780008720a900ee
:1083a800004006008740a900004006007546880086
:1083b800c5498000750c8800d5498000a50c880047
:1083c800a5498000150c8800b5498000450c880037
:1083d80025002000250c88007546800084e0a9004f
:1083e800004006000c28ae00070037000c28a90042
:1083f8007228ef002fe1a9008a00a9002621ef00ca
:108408002fe1a800004006002fe1a9008a00a9007a
:108418002621ef008900a9009900a8000040060065
:108428004029ef006e89ae004449a8000c48af000f
:108438004449a90089e0a9000040060021e3a900f9
:108448002043a9008de3a90085c0a90085a0a90043
:108458000040060005002400b5017800725780002e
:10846800440120000410b900030040000180b0005e
:1084780053012000110009004308d80070578800f4
:1084880060488800b50178008257800044012000c8
:108498000410b900030040000180b000530120001f
:1084a800110009004308d8008057880090488800c8
:1084b800b5017800a341880003007800030120007b
:1084c800110009000380d800b0418800b501780088
:1084d80062578000440120000410b90003004000e6
:1084e8000180b00053012000110009004308d800a2
:1084f8006057880050488800b5017800f243800032
:108508007410b900030040000180b000530120003e
:10851800110009004308d800f0438800d326200042
:1085280003005000e0438800b501780073418800db
:108538000300780003012000110009000380d8001f
:1085480080418800b5017800b5017800d2438000e9
:108558007410b900030040000180b00053012000ee
:10856800110009004308d800d0438800c0438800a0
:10857800b5017800b5017800b5017800d3418800cd
:108588000300780003012000110009000380d800cf
:10859800e0418800b501780085a0a9000000060028
:1085a800d04480003c69af00a05180000301200046
:1085b8000300b90043062000110009004308d80051
:1085c80080448800f0448000030120000300b900c3
:1085d80043062000110009004308d8009044880091
:1085e80010458000030120000300b9004306200065
:1085f800110009004308d800a044880030458000d5
:108608003c49af00d0518000030120000300b900ad
:1086180043062000110009004308d800b044880030
:1086280050458000030120000300b90043062000e4
:10863800110009004308d800c04488000000060063
:10864800010020009101880001c024001100ba0037
:10865800f2ff2f0002016800110032006043880019
:108668000208200081004100020025000288e7007e
:10867800f6ff370002082000828050003100ba005f
:108688006294200037000800030000000000eb009f
:108698003100ba0000197800000000000000060050
:1086a80002082000828050003100ba006294200045
:1086b80037000800030000000000eb003100ba009a
:1086c80000197800000000000000060001002000ea
:1086d8009101880001c024001100ba00f2ff2f00a8
:1086e800020168001500320060438800020820007b
:1086f80081004100020025000288e700f6ff3700ec
:1087080002402000828050001100ba000000e800fa
:1087180060438800ae43020000000000624380000e
:1087280010002400003b880003002000930188000b
:10873800ce430200000000000000060010002400e4
:10874800003b880062438000ce4302000000000026
:108758000000060020042400003b880003002000dd
:10876800930188008108bb000500fc00500520002b
:10877800303b8800a20a2000323b880061e7a8004d
:10878800000000000000000061e7af00feff3700b6
:1087980000000600020078008008bb008098bb003b
:1087a8006294200037000800040000000000eb007d
:1087b800320078008008bb008098bb0000000000f1
:1087c800000000000500fc0050052000303b880038
:1087d800a10a2000313b880061e7a80000000000e2
:1087e8000000000061e7af00feff37000000060050
:1087f8000000000001000000040000000700000065
:108808000b0000000e000000110000001400000022
:10881800170000001b0000001e00000021000000df
:1088280025000000280000002b0000002f00000099
:1088380033000000360000003a0000003e0000004f
:1088480042000000460000004a0000004e00000000
:1088580052000000570000005b00000060000000ac
:10886800650000006b00000070000000760000004a
:108878007c00000082000000880000008f000000db
:10888800970000009f000000a7000000af00000054
:10889800b9000000c3000000ce000000da000000ac
:1088a800e7000000f50000000401000016010000c8
:1088b800290100003e01000056010000710100007e
:1088c80091010000b7010000e30100001802000058
:1088d8005a020000ad0200001a030000af030000b6
:1088e80087040000e105000069080000270f000068
:1088f800245000004d5400004b3300003134000078
:108908002c3000002c3100002c3100002c310000ec
:108918002c3000002c3000002c3000002c300000df
:108928002c3000002c3000002c3000002c300000cf
:108938002c3000002c3000002c3000002c300000bf
:108948002c3000002c3000002c3000002a320000af
:10895800390d00000a000000245000004d540000aa
:108968004b320000353100002c350000373600004e
:10897800303000002a320000430d00000a000000d9
:10898800245000004d5400004b32000032300000eb
:108998002c320000303000002a320000430d000065
:1089a8000a000000245000004d5400004b35000020
:1089b800303000002c320000303000002c30000035
:1089c8002c3000002c3000002c3000002a31000030
:1089d800410d00000a000000245000004d54000022
:1089e8004b330000303000002c32000030300000e3
:1089f8002c3000002c3000002c3000002c300000ff
:108a08002a310000430d00000a000000244700003e
:108a180050560000544700002c310000393800003f
:108a28002e390000372c0000542c00002c4d00007b
:108a38002c3000002e320000313300002c4e000094
:108a48002c3000002e330000393400002c4b00007d
:108a58002c4100002a330000440d00000a000000e9
:108a68002447000050470000474100002c30000018
:108a78003131000035320000382e0000303000005f
:108a8800302c000031380000323700002e31000051
:108a98003931000030300000302c00004e2c00002e
:108aa8003036000039350000372e00003636000019
:108ab80030300000303000002c5700002c3100000e
:108ac8002c3700002c3000002e390000382c000014
:108ad8002d310000382e000033310000392c000001
:108ae8004d2c0000313700002e38000030360000d1
:108af8002c4d00002c2c00002a360000460d0000ea
:108b08000a00000024470000505200004d430000b6
:108b18002c3000003533000037340000302e0000c0
:108b280030300000302c0000412c000032350000ad
:108b3800303300002e36000033310000392c00009d
:108b48004e2c00003132000031330000362e000078
:108b580030300000393900002c4500002c3200006c
:108b68002e360000392c0000373900002e36000060
:108b7800352c000031300000303100003036000064
:108b88002c2c00002c4100002a350000330d000079
:048b98000a000000cf
:020000040000fa
:108b9c0000080000140700000000000000000000a6
:020000040000fa
:048bac000000fe00c7
:00000001FF
